:1000000018550020F12600009D69000021270000FE
:100010002127000021270000212700000000000008
:10002000000000000000000000000000D9250000D2
:10003000212700000000000091250000DB6800007F
:10004000C9260000C9260000C9260000C9260000F4
:10005000C9260000C9260000C9260000C9260000E4
:10006000C9260000C9260000C9260000C9260000D4
:10007000C9260000C9260000C9260000C9260000C4
:10008000C9260000C9260000C9260000C9260000B4
:10009000C9260000C9260000C9260000C9260000A4
:1000A000C9260000C9260000C9260000C926000094
:1000B000C9260000C9260000C9260000C926000084
:1000C000C9260000C9260000C9260000C926000074
:1000D000C9260000C9260000C9260000C926000064
:1000E000C9260000C9260000C9260000C926000054
:1000F000C9260000C9260000C9260000C926000044
:1001000053B94AB9002908BF00281CBF4FF0FF317E
:100110004FF0FF3000F06CB9ADF1080C6DE904CE82
:1001200000F006F8DDF804E0DDE9022304B07047D2
:100130002DE9F047089E0D4604468E46002B40F000
:1001400082808A42174646D9B2FA82F24AB1C2F197
:10015000200105FA02F320FA01F1974041EA030E6B
:1001600094404FEA1748230CBEFBF8FCB9B208FBD9
:100170001CEE43EA0E430CFB01F098420AD9FB182F
:100180000CF1FF3580F01681984240F21381ACF1FA
:10019000020C3B441B1AA4B2B3FBF8F008FB10336B
:1001A00044EA034400FB01F1A14209D93C1900F1E2
:1001B000FF3380F00181A14240F2FE8002383C44CE
:1001C000641A40EA0C4000211EB1D4400023C6E965
:1001D0000043BDE8F08702B9FFDEB2FA82F2002ADE
:1001E0004FD1CB1B4FEA174E1FFA87F80121B3FB03
:1001F000FEFC250C0EFB1C3345EA034508FB0CF303
:10020000AB4207D97D190CF1FF3002D2AB4200F2AC
:10021000E7808446ED1AA3B2B5FBFEF00EFB105545
:1002200043EA054408FB00F8A04507D93C1900F152
:10023000FF3302D2A04500F2D7801846A4EB080491
:1002400040EA0C40C0E78B4208D9002E00F0AF8096
:100250000021C6E900050846BDE8F087B3FA83F13E
:1002600000294BD1AB4202D3824200F2B780841AFC
:1002700065EB030301209E46002EAAD0C6E9004E7E
:10028000A7E7C2F1200C01FA02F3974020FA0CF024
:100290004FEA174E21FA0CFC1843BCFBFEF1050C8B
:1002A0000EFB11CC1FFA87F845EA0C4501FB08F359
:1002B000AB4204FA02F409D97D1901F1FF3C80F048
:1002C0008B80AB4240F2888002393D44EB1A85B204
:1002D000B3FBFEF00EFB103345EA034500FB08F3C9
:1002E000AB4207D97D1900F1FF3C71D2AB426FD907
:1002F00002383D44EB1A40EA014178E7C1F1200C95
:100300008B4022FA0CF71F4320FA0CF405FA01F394
:100310004FEA174E25FA0CF51C43230CB5FBFEF9EA
:100320001FFA87F80EFB195543EA054509FB08FA41
:10033000AA4502FA01F200FA01F308D97D1909F180
:10034000FF3047D2AA4545D9A9F102093D44A5EBA2
:100350000A05A4B2B5FBFEF00EFB105544EA0544B5
:1003600000FB08F8A04507D93C1900F1FF352DD254
:10037000A0452BD902383C4440EA0940A4EB0804CC
:10038000A0FB02894C45C6464D4619D316D05EB136
:10039000B3EB0E0264EB050404FA0CFCCA404CEA11
:1003A0000202CC40C6E900240021BDE8F0873146B6
:1003B00030460EE7AC46EDE6184601E74345E6D287
:1003C000B8EB020E69EB07050138E0E72846D3E7F2
:1003D00060468FE78146BAE7614677E708464BE714
:1003E000ACF1020C3D4415E702383C4426E700BF5F
:1003F000704700BF30B585B04FF00000032363F3B2
:1004000002006FF3C500324B324A9B1AC3F3C90393
:1004100063F38F10304905F0EDFF00F09BF82F4893
:1004200000F068F8A8B101A800F0B0FD10B34FF0DB
:100430000000012363F302006FF3C500244B254A3B
:100440009B1AC3F3C90363F38F10254905F0D2FF4C
:10045000FEE7012363F302006FF3C5001C4B1D4A46
:100460009B1AC3F3C90363F38F101C4A1D4905F09F
:10047000C1FFFEE703254FF0000065F302006FF3B4
:10048000C500134C134BE41AC4F3C90464F38F1072
:10049000039A154905F0AEFF4FF0000065F3020026
:1004A0006FF3C50064F38F10104905F0A3FF01A896
:1004B00004F036FE4FF00000012363F302006FF3F7
:1004C000C50064F38F100A4905F094FFFEE700BFF2
:1004D000F08E0000E88E0000588F00006C8F000046
:1004E0009C8F0000808F0000BC8F0000E88F000010
:1004F0000890000008B5054B1B6813B1034B186842
:1005000008BD04F033FB014B1860F7E790010020B1
:1005100010B900200860704708B502464FF000008F
:10052000012363F302006FF3C500074B07495B1A11
:10053000C3F3C90363F38F100023054905F05AFF85
:100540006FF0150008BD00BFF08E0000E88E0000BF
:100550002890000008B54FF4C051024803F096FD02
:1005600008BD00BF9401002070B5A4B0202928D890
:1005700006460D460024144B1B68A3421CDD09A847
:1005800008F0BCF9002109A803F0AEFE0F4B03EB05
:10059000C4025268126853F8341009A808F0B4F97C
:1005A00001A909A808F0F3F92A46314601A806F086
:1005B0005FFA18B10134DEE74FF0FF34204624B073
:1005C00070BD4FF0FF34F9E74C90000050900000F0
:1005D0002DE9F041D6B014461D465F9E04965E9EFE
:1005E000039606AE02965D9E01965C9E009604F010
:1005F000DAFD0646002840F08280609B23B120226D
:1006000006A9184606F04BFA002300934FF6FF7335
:100610002A4621464EA804F005FE064600286ED163
:10062000074680464FF0FF341DE04FF0FF341AE0DC
:100630004FF0FF3417E04FF0FF34012713E0BDF80F
:100640005231202B5FD10EAA5599284605F0CBFFD9
:1006500000285BD120220EA906A806F009FA00287E
:1006600056D14FF0010854AB0DF5A97255A94EA80B
:1006700004F03DFE002840DB38DCBDF85021102A94
:10068000DDD0012A21D0202AEDD1002CCDDB294B51
:100690001B68A342CCDDBDF85231B3F5807F3FD15A
:1006A0000EAA5599284605F09EFF00283BD1E4B2DA
:1006B0000094BDF852310EAA202106A800F0AEF831
:1006C0000028B8D04FF0FF34CDE7BDF85231202BD1
:1006D00021D80EAA5599284605F085FFF0B99DF856
:1006E00052110EA8FFF740FF0446BCE7B8F1000F17
:1006F0001CD027B94FF0FF3601E04FF0FF363046EF
:1007000056B0BDE8F0814FF0FF36F8E70646F6E751
:100710004FF0FF36F3E74FF0FF36F0E70646EEE71F
:100720004FF0FF36EBE74FF0FF36E8E74FF0FF36CC
:10073000E5E700BF4C90000070B5ADF51C7D0E469E
:1007400019464368B3F5807F51D1202A52D141AA7E
:1007500003F088FD054600284FD19DF80332BC2BDD
:100760004ED10DF2E31109A804F06FFE2B46DE2BEB
:1007700007DC41AAD25C09A8C45C6240C2540133C0
:10078000F5E79DF8243003F07F038DF82430BD2D6C
:1007900004DC09AB5B5DB3BB0135F8E79DF8E230E3
:1007A000012B35D181A808F0A9F8002181A803F018
:1007B0009BFD0822184981A808F0A6F8202231469E
:1007C00081A808F0A1F820220DF1E30181A808F02A
:1007D0009BF801A981A808F0DAF820220DF2E311B4
:1007E00001A806F045F980B14FF0FF300DE04FF061
:1007F000FF300AE04FF0FF3007E04FF0FF3004E039
:100800004FF0FF3001E04FF0FF300DF51C7D70BD63
:100810004FF0FF30F9E700BF589000002DE9F0439A
:10082000ADB006460F4690461D469DF8D09000227A
:10083000114601A808F01CF8114C54F83930009307
:1008400004EBC904626812681A44694601A804F0FE
:10085000AAFD044610B9029BAB4206D001A808F0DD
:1008600015F820462DB0BDE8F08343463A463146A0
:1008700001A8FFF761FF044601A808F007F8F0E7B8
:100880005090000008B51022034906F0F1F808B1B5
:10089000022008BD0120FCE7AC90000070B586B0D6
:1008A0000D460123ADF80430002407E0286805F068
:1008B00099FE23E0286805F095FE0134012C1BD831
:1008C000294606AB234413F8140C01F031FB06460D
:1008D000A0B928688168102302AA103905F083FEA8
:1008E00006460028E2D11022064902A806F0C0F808
:1008F00006460028DED101E04FF0FF36304606B054
:1009000070BD00BFAC90000008B581681023044A98
:10091000103905F087FE00B908BD0120FCE700BFD3
:10092000AC90000030B585B002A9012004F08FFE24
:1009300000286ED16946022004F089FE00286AD1A1
:10094000002407E02B79042B29D09DF80A2093423C
:1009500025D00134022C48D804EB44032F4A02EB83
:1009600043059DF8081012F8130004F0E1FD00287B
:10097000EFD09DF80010687804F0DAFD0028E8D088
:10098000AB78042B03D09DF80B209342E1D1EB7898
:10099000042BD7D09DF803209342DAD1D2E74FF051
:1009A0000000032363F302006FF3C5001C4B1D4AD4
:1009B0009B1AC3F3C90363F38F106B79022B07D023
:1009C000032B10D0042B01D0174A02E0174A00E095
:1009D000174A184905F00EFD6879831EDBB2022B19
:1009E00015D9FF2013E0144AF3E74FF0000003236A
:1009F00063F302006FF3C500094B0A4A9B1AC3F365
:100A0000C90363F38F100D4905F0F4FC012005B014
:100A100030BDFF20FBE7FF20F9E700BFBC900000DE
:100A2000F08E0000E88E00007090000084900000BE
:100A3000609000008C900000689000009C90000086
:100A400002680E4B9A420DD1C2680389D843824294
:100A50000CD810B4D418012010B18B68A34203D96C
:100A600010BC7047002070470020F9E7002010B14B
:100A70008B68A34200D97047002070473DB8F396B9
:100A800000B587B0134600200490039002904FF405
:100A900080720192054A00920A460146FFF798FDCE
:100AA00010B907B05DF804FB0320FAE7F425002035
:100AB0002DE9F04182B006460C461546002004F0B0
:100AC00052FB01A9C0B201F033FA28B14FF0FF3553
:100AD000284602B0BDE8F0812C2000FB04672146C7
:100AE000304604F070FE00B33B6913F0100F1CD1C8
:100AF000DDF8048041463846FFF7A2FF00BB4CBB3F
:100B00004FF00000012363F302006FF3C500154BA3
:100B1000154A9B1AC3F3C90363F38F1004BB134A2E
:100B2000134905F067FC012501E024B9012501986E
:100B300005F058FDCCE70199304604F04CFFF5E78D
:100B40002B46424639463046FFF79AFF05460028B5
:100B5000EDD0D4E701988268002105F093FDCFE73E
:100B6000044ADDE7F08E0000E88E0000DC90000013
:100B7000E4900000D090000030B583B005460C46EC
:100B8000002300930193084604F0BCFE30B32A68AA
:100B90001F4B9A4216D0EA6A1D4B9A4218D0019B0D
:100BA000009A934200D90093009BA360009A2146CB
:100BB000284600F0B3FC174B1A68002A16DC002008
:100BC00003B030BD6A460021284604F0A5FDE2E7E7
:100BD00001AA0121284604F09FFDE0E704F1080185
:100BE000002004F049FDA3680093DFE74FF0000008
:100BF000022363F302006FF3C500074B07495B1A3A
:100C0000C3F3C90363F38F10054905F0F3FBD6E77F
:100C10003DB8F396F4260020F08E0000E88E000028
:100C20000891000038B504460D46FFF7A5FF0246BF
:100C3000EB7984F85830033BDBB2012B0CD9EB790C
:100C4000022B13D0042B11D0032B0FD094F8583063
:100C5000FF2B15D0104638BD002004F062FF02467D
:100C60000028ECD0FF2384F85830E8E7002004F097
:100C700045FF02460028E9D0FF2384F85830E5E715
:100C80004FF00000012363F302006FF3C500054B32
:100C9000054A9B1AC3F3C90363F38F10034905F098
:100CA000A9FBFEE7F08E0000E88E00003491000002
:100CB00038B504460D4604F0CEFD68B90022114651
:100CC000204604F0DEFDE8B9204600F0E1FA78BBEA
:100CD000012384F8583014E04FF00000022363F33E
:100CE00002006FF3C500474B474A9B1AC3F3C90381
:100CF00063F38F108022454905F07CFB012384F8C3
:100D0000583038BD4FF00000022363F302006FF348
:100D1000C5003C4B3C4A9B1AC3F3C90363F38F10D5
:100D200000223B4905F066FB012384F85830E8E7D0
:100D3000284604F0DDFD2946204604F0A6FEE8B969
:100D4000284604F0DFFD80F001012A46C9B22046A2
:100D500004F097FD40BB284604F0D4FD002839D0AC
:100D6000EB79012B43D02A4601212046FFF7A0FE54
:100D7000002843D0052384F85830C2E74FF0000024
:100D8000022363F302006FF3C5001E4B1E4A9B1A39
:100D9000C3F3C90363F38F1000221E4905F02AFB39
:100DA000012384F85830ACE74FF00000022363F3CE
:100DB00002006FF3C500134B134A9B1AC3F3C90318
:100DC00063F38F100022124905F014FB012384F80D
:100DD000583096E729462046FFF724FF2A4600218F
:100DE000204604F04EFD012384F8583089E7294657
:100DF000204604F061FD84F8580082E7EB7984F81E
:100E000058307EE7F08E0000E88E00003C91000034
:100E10007C910000A49100002DE9F84F884691468E
:100E20001F46DDF828A00B9E00250FE023460F4A41
:100E3000E919404605F0D7FBA0B923460B4A05EB5C
:100E40000A01484605F0EEFB70B92544B54206D2CA
:100E5000741BB4F5806FE9D94FF48064E6E7002095
:100E6000BDE8F88F0120FBE70120F9E7F419002025
:100E700070B584B004460D466022002105F033FEB3
:100E80003D4B63623D4B236500260CE0314600205C
:100E900004F069F92C2101FB06F120312144C0B294
:100EA00001F046F80136012EF0D969462046FFF7D9
:100EB000FFFE94F858308DF80730042B25D8022B0C
:100EC0002ED2012B31D194F85830FF2B31D0012B89
:100ED00006D06A460021204604F0D3FC064690B9AD
:100EE000002211462046FFF7E3FD064698BB10227C
:100EF0000021684605F0F7FD236A5B782B71236AB1
:100F00005B68AB602C60002530E0052B0DD1002024
:100F100004F007FE0028D6D0FF2384F85830D2E72B
:100F20006946204604F0FFFCCDE7FF2384F85830E3
:100F3000C9E74FF00000012363F302006FF3C5001F
:100F40000F4B104A9B1AC3F3C90363F38F100E496A
:100F500005F050FAFEE70326D5E7C5F101032C2280
:100F600002FB0343186A05F03DFB0135012DF4D95E
:100F7000304604B070BD00BFF41D0020F4210020F5
:100F8000F08E0000E88E00003491000008B50146A4
:100F90000148FFF76DFF08BD941900202DE9F043CB
:100FA00083B00F4615461C46DDF82880536A53F877
:100FB00030601A68B61A013853F83030A3EB0209D2
:100FC0002368012B1BD03A463146404604F0FFFC13
:100FD000019700964B46424641462846FFF71CFFC4
:100FE0002146284604F0C0FC23680133236018B171
:100FF0000C4A13680133136003B0BDE8F083E36863
:10100000022B04D10B99284604F0E5FCDBE74146AE
:10101000284604F0E0FC22464146284604F013FD31
:10102000F0E700BFF42600202DE9F04383B00E4620
:1010300015461C46526A52F830101368A1EB03089B
:10104000013852F83070FF1A2A6D52F830101368C8
:10105000A1EB03092379012B05D02379022B1CD0A6
:1010600003B0BDE8F083324639460A9804F0AFFC7D
:10107000019600974B460A9A0B992846FFF7CCFE3B
:101080002146284604F070FC022323710028E4D096
:10109000114A136801331360DFE7324649460B9863
:1010A00004F095FC0196CDF8009043460B9A0A99FE
:1010B0002846FFF7B1FE2146284604F055FC236878
:1010C00001332360012323710028C9D0024A136829
:1010D00001331360C4E700BFF426002070B582B06E
:1010E00015461E46002B36D0436A5C687379012B87
:1010F00011D0022B17D00024002004F034F801A9ED
:10110000C0B200F015FF68B30124019805F06AFA37
:10111000204602B070BD01BB32681C4B1B689A426E
:10112000EAD80024E8E73368012B07D9174A126888
:10113000934203D899B900240121DDE7012B01D0A6
:101140000024D9E701B100240129D5D13379022B3C
:10115000D2D10021D0E70024CEE70024CCE7002440
:101160002146C9E720232A462146019805F03BFA8B
:10117000044640B9002EC8D02A68054B9A42C4D014
:101180004FF0FF34C1E70124BFE700BF000000209B
:101190003DB8F3962DE9F04F85B006460D46019215
:1011A0000146002004F0DCF9041E62DBD5F85CA0E7
:1011B000304604F0E0F981464FF0000B01274FF074
:1011C000FF3805E0874201D00BF1010B2C460746A2
:1011D000002C13DD651E5FFA8AF101230DF10F0269
:1011E00005FB0191304603F0CAFF002843DB0128CC
:1011F000E8D0B8F1FF3FE9D1A046E7E7BBF1010F26
:101200000EDCB8F1FF3F3AD0B8F17F0F1ADC0123B2
:1012100001994B7108EB03020A600B7100202BE06F
:101220004FF00000012363F302006FF3C500154B7C
:10123000154A9B1AC3F3C90363F38F10134905F0D2
:10124000D9F8DEE70223019A5371A8F1800808EB70
:10125000D8735B1001331360B8F1000F08F0010878
:10126000B8BFC8F1000808F1010882F80480002026
:1012700002E0072000E0012005B0BDE8F08F00206B
:10128000FAE700BFF08E0000E88E0000CC9100006D
:1012900038B5856A446DA54202D0631CAB4211D1BA
:1012A000802D22D800231946A34244D2426A02EB81
:1012B000C3025168026D02EBC30252688A4227D111
:1012C0000133F1E74FF00000022363F302006FF3F4
:1012D000C500284B284A9B1AC3F3C90363F38F1038
:1012E000264905F087F8002024E04FF00000022393
:1012F00063F302006FF3C5001E4B1F4A9B1AC3F332
:10130000C90363F38F101E4905F074F8002011E043
:101310004FF00000022363F302006FF3C500154B8A
:10132000154A9B1AC3F3C90363F38F10154905F0DF
:1013300061F8002038BDA5421AD9426A02EBC30306
:101340005B68994201D10120F4E74FF000000223CD
:1013500063F302006FF3C500064B074A9B1AC3F301
:10136000C90363F38F10074905F044F80020E1E753
:101370000120DFE7F08E0000E88E0000EC91000015
:10138000209200004C92000010B586B004A9012004
:1013900004F05DF94FF00000032363F302006FF3E4
:1013A000C500264B264A9B1AC3F3C90363F38F106B
:1013B0009DF81030012B2DD0032B29D0214B9DF807
:1013C00011209DF812109DF8134002940191009293
:1013D0001D4A1E4905F00EF89DF81030012B03D16F
:1013E0009DF81230032B17D04FF00000032363F356
:1013F00002006FF3C500114B114A9B1AC3F3C903D6
:1014000063F38F10124904F0F5FF002006B010BD01
:10141000104BD4E7104BD2E74FF0000063F302000B
:101420006FF3C500054B064A9B1AC3F3C90363F368
:101430008F100A4904F0DEFF0220E7E7F08E00007B
:10144000E88E0000749200008892000098920000DC
:10145000F09200008092000078920000D492000088
:10146000F0B587B00C46496801F0FF21234DA94231
:1014700004D1064617462268012A01D007B0F0BD04
:1014800004A9184604F0E3F84FF00000032363F3C7
:1014900002006FF3C5001A4B1A4A9B1AC3F3C90323
:1014A00063F38F109DF81030012B24D0032B20D034
:1014B000154B9DF811209DF812109DF813500295C0
:1014C00001910092114A124904F094FF9DF81030E6
:1014D000032BD3D13946304604F07DFA384604F068
:1014E000EDF8A168384604F002F93846FFF70CFA27
:1014F000C4E7084BDDE7084BDBE700BF0001000451
:10150000F08E0000E88E000074920000049300004A
:10151000989200008092000078920000F0B585B0AB
:1015200007460D4600243E4B1C60436A5E68344407
:101530003B490B6801330B609442F8D3284604F012
:10154000E1F970B1F86D04F006F8BA6A013A0023C7
:101550003344984201D9013AFAE7314B1B68934270
:1015600014D203A9012000F0E3FC02A9022000F03C
:10157000DFFC0223029A29463846FFF771FF6B7998
:10158000012B17D002236B71012438E04FF00000CB
:10159000022363F302006FF3C500224B224A9B1A19
:1015A000C3F3C90363F38F10204904F023FF012321
:1015B000EB7132E01A4B1C680AE0029B0193039B1B
:1015C00000932B463A4631462046FFF7E7FC013CA4
:1015D0003CB12A68124B1B689B1A01339C42F6D817
:1015E000EBE701232B60CDE7029B0193039B009364
:1015F0002B463A4631462046FFF716FD0134084B8C
:101600001B68A34203D32B68A342F7D8ECE70398E7
:1016100004F0E8FF029804F0E5FF05B0F0BD00BF5C
:1016200000000020F08E0000E88E000014930000FF
:10163000BFF36F8F72B6002308E003F120010B4A5D
:101640004FF0FF3042F821000133DBB2072BF4D911
:10165000002308E003F16001044A4FF0FF3042F834
:1016600021000133DBB2072BF4D9704700E100E021
:101670002DE9F04F89B092469B469DF84C3001937E
:101680009DF85070142400970F460646129D5AEAA2
:101690000B0318D04FEAE5792A464B465046594687
:1016A000FEF72EFD274B13441A7808AB234403F8AA
:1016B000182C2A464B4650465946FEF721FD8246D5
:1016C0008B46013CE3E735463E46009F142C0BD089
:1016D0000134159B04EB0308B8F1150F0AD0A8F1EB
:1016E0001508A146019C0FE0302208AB234403F803
:1016F000182CEEE74FF00008A146019C04E03146AB
:101700003846A84708F1FF38B8F1000F03DD002C78
:10171000F5D14C4600E04C46142C07D808AB2344C6
:10172000314613F8180CA8470134F5E7B8F1000F5B
:1017300005DD31463846A84708F1FF38F6E709B01D
:10174000BDE8F08F5494000008B50B6801330B60BE
:10175000014B1B68984708BD04000020014B18602E
:10176000704700BF0400002000B583B002460B465E
:101770000021019101A9034804F062FA03B05DF869
:1017800004FB00BF491700002DE9F04383B0044675
:1017900008461546238B13F0080F05D103F0070602
:1017A00000230093019369E0012909D043F020034D
:1017B000238385F31188BFF36F8F03B0BDE8F083F7
:1017C00043F010032383F4E7204604F0EEFB57E0D8
:1017D000D4F814904A466946204604F0FFFB0027DF
:1017E0005AE023691F680621204604F0B7FB4FF03A
:1017F000000951E023695F680421204604F0AEFB34
:101800004FF0000948E023699F680521204604F055
:10181000A5FB4FF000093FE0002246E0002244E033
:1018200043F00803238385F31188BFF36F8F0029EA
:1018300044D1009B2BB14B4642466946204604F0FA
:1018400043FC17B125492046B8474FF02003EFF37A
:10185000118583F31188BFF36F8F238B23F0080367
:101860002383238B13F0100F2ED023F01003238338
:101870000120268B06F0070600289AD00228A3D064
:10188000002896D00128A3D00328AAD00428B1D0DC
:101890000528B8D00027B946238B03F00708B045C8
:1018A000BAD0A268002AB9D001221146002AB7D1C5
:1018B000009A002AB4D1002FB2D1D2E74A4641465D
:1018C000204604F053FBB4E713F0200F04D023F0BC
:1018D000200323830220CCE70020CAE7F760000042
:1018E0002DE9F04385B080460F461546124B1B6824
:1018F00098470646002400E00134104B104A9B1A1A
:10190000B4EB231F15DA0E4800EB041043685B7933
:10191000002BF1D003952301094AD358D3F8049042
:10192000B9F1000FE8D000953B4632464146C84722
:10193000E2E705B0BDE8F08308000020388F000022
:10194000188F000008B5044B044A1A604FF4004099
:1019500000F00EFA08BD00BF08000020ED63000093
:10196000054B064A9B1AB1EBD30F02D252F8310055
:1019700070470020704700BF188F0000E88E0000FD
:1019800008B50B4BC31A1B1101334268137143682E
:101990001960436801225A71064B1B781BB1054B35
:1019A00001221A7008BD044803F006FBF7E700BFE8
:1019B000188F0000082D0020F400002038B5154BCA
:1019C000BFF35B8F53E8002F511C43E80010002841
:1019D000F8D1BFF35B8FDAB9002405E004220021BF
:1019E0002846FFF7CDFF01340B4B0C4A9B1AB4EB92
:1019F000231F0DDA094D05EB04152B7B002BF2D0CC
:101A00002301064AD3585B69002BE7D09847E5E7E6
:101A100038BD00BFF8260020388F0000188F000066
:101A2000104B1B7803B1704710B5FFF7C7FF0024B8
:101A300000E001340C4B0D4A9B1AB4EB231F0CDA67
:101A40000A4800EB041043685B79002BF1D02301B6
:101A5000064AD3581B699847EBE7024B01221A70DC
:101A600010BD00BF092D0020388F0000188F000026
:101A70000EB400B582B0014603AB53F8042B0193BA
:101A8000044804F0DDF8002002B05DF804EB03B078
:101A9000704700BF1D640000F0B585B011F0440F21
:101AA00005D01A4B1C6834B9002005B0F0BD1849A8
:101AB000FFF7DEFFF9E7174B1968B2FBF1F1B1FB55
:101AC000F4F5154AA2FB0532D20A4FF4616606FB13
:101AD0001256124BA3FB06735B0904FB15114FF45E
:101AE0007A7505FB01F1B1FBF4F707FB141105FB57
:101AF00001F1B1FBF4F402940197C3EB0311A6EBDF
:101B0000810100910649FFF7B3FFCEE7FC260020D4
:101B10006894000000270020C5B3A29189888888B6
:101B20007494000061B108B52AB1064A52F8232026
:101B300012B9054A00E0044A0449FFF799FF08BDBD
:101B4000704700BFEC94000090940000989400004F
:101B500011F0100F0BD108B511F0200F03D004497C
:101B6000FFF786FF08BD0349FFF782FFFAE77047DA
:101B7000909600009C9400002DE9F04105460F4628
:101B8000164698460699FFF7E3FF0024444505DA18
:101B900023492846FFF76CFF0134F7E7002409E0EA
:101BA0001F492846FFF764FF0BE01E492846FFF750
:101BB0005FFF01340F2C0CDC002C02DD14F0070F4A
:101BC000EED0B442F1D23A5D17492846FFF750FFF4
:101BD000EFE716492846FFF74BFF002409E01049BC
:101BE0002846FFF745FF0BE011492846FFF740FF65
:101BF00001340F2C12DC002C02DD14F0070FEED0A4
:101C0000B44206D23A5DA2F120035E2BECD92E221B
:101C1000EAE703492846FFF72BFFE9E7BDE8F08133
:101C2000C4940000A8940000A0940000AC940000AC
:101C3000B0940000F8B5044616461D4649B9002781
:101C400086B10123079A934013F0100F16D10C4E62
:101C500009E00C4B079A53F822200B49FFF708FFC5
:101C60000746EDE7064E06992846FFF779FE02463D
:101C700031462046FFF7FCFE3844F8BD034EF2E73C
:101C8000B494000000950000C0940000BC940000D3
:101C900070B584B005461E46C1F3C203C1F3891076
:101CA00011F007040FD1089B32462946104803F073
:101CB000C7FF94B9304604F0CBFB98B10D492846D4
:101CC000FFF7D6FE0EE00290019300941346012226
:101CD0000999284604F0DFFBE5E7224609992846E2
:101CE00004F0CDFB284604F0FDFB04B070BD00BF3E
:101CF0001D640000C89400002DE9F04784B0074639
:101D00001D460C9E0D9CDDF8388001F0070AC1F3DA
:101D1000C203C1F3891102910193CDF800A01346CB
:101D20000122414604F0B7FB81462A460F49384656
:101D3000FFF79EFE74B12546102C28BF1025CDF864
:101D400000804B462A4631463846FFF715FF2E44A1
:101D5000641BEFE752464146384604F090FB384694
:101D600004F0C0FB04B0BDE8F08700BF9894000009
:101D7000074B01221A60074B984205D94008044AD4
:101D800013685B001360F6E7034B1860704700BFF1
:101D90000027002040420F00FC26002008B5034821
:101DA00002F0E4FE024B586008BD00BF149500002D
:101DB0000C27002008B5024804F094FB08BD00BFC2
:101DC0004895000000B585B00F200290079801905B
:101DD000069800900248FFF78FFF05B05DF804FBFE
:101DE0004895000000B583B00F2001900498009042
:101DF0000248FFF74DFF03B05DF804FB4895000073
:101E0000014B01221A7070470B2D002008B518B93C
:101E1000044B00221A7008BD41F2883006F014FF0E
:101E2000F9E700BF0B2D002038B504460A4B01220C
:101E30001A700A4B1B7803B938BD002000F07EFBF6
:101E40000028F9D0044B1B78002BF5D0651E2046E6
:101E5000FFF7DCFF2C46F0E70B2D00200C2D0020B7
:101E6000F8B506460D46042706E03846FFF7DCFFC6
:101E70009CB90D4B1B7883B12A463146002000F0F7
:101E8000F9FA04460028F0D1074B1B78002BEFD05D
:101E9000013F3846FFF7BAFFEAE714B9024B1B7857
:101EA00003B92C462046F8BD0B2D002008B5034B86
:101EB00001221A70024804F015FB08BD0C2D002009
:101EC0008095000000B585B00F2002900798019022
:101ED000069800900248FFF70FFF05B05DF804FB7D
:101EE0008095000000B583B00F2001900498009009
:101EF0000248FFF7CDFE03B05DF804FB80950000BB
:101F000010B404460023084A12689A4209DD1A01F7
:101F10000649096801EB03108A5CA24202D0013332
:101F2000F1E7002010BC7047E09500000C00002095
:101F3000084B1B683BB110B50C46FFF7E1FF28B119
:101F40002060002010BD6FF00C0070476FF00100A2
:101F5000F8E700BF0C00002000B58BB003AB009386
:101F6000024B04F018FB0BB05DF804FB5B6500004E
:101F700010B504460A2807D0074B1868E1B28368F9
:101F80005B689847204610BD034B186883685B6800
:101F90000D219847F0E700BF3027002010B5044C12
:101FA000204600F0B9FD2046FFF7D8FB10BD00BF6A
:101FB000711F000008B5044802F0D8FD034B1860FB
:101FC000FFF7ECFF002008BD14950000302700202B
:101FD000014B01221A6070470800004082B0054B97
:101FE00000221A601B680193019B034B01221A60B7
:101FF00002B07047040100400C00004082B0054B65
:1020000000221A601B680193019B034B01221A6096
:1020100002B070470001004004000040014BD86846
:10202000403070475C00002010B54FF02003EFF304
:10203000118483F31188BFF36F8F134A136843F041
:102040000203136013F0010F10D04FF08043D3F858
:102050000C24D3F80C3412F0010F01D1002306E058
:10206000FFF7DCFF04F0B9FB012300E0002384F359
:102070001188BFF36F8F13B904F0D4FB10BD00219A
:10208000024804F0BDFBF9E7942700205C00002023
:10209000034BDB68C01A8010024B03FB00F0704753
:1020A0005C000020B76DDBB638B505460C46FFF77F
:1020B000EFFF01464022034804F0B9FB01462846E1
:1020C000A04738BD5C00002030B585B005460C4601
:1020D00000230193084B02930391FFF7D9FF0146B8
:1020E000402301AA054804F0BCFB011E01DB05B03A
:1020F00030BD2846A047FAE7AF6800005C0000202A
:1021000008B501214FF4807004F0F3FA60B10021AA
:102110000E4804F00EFB836813F0070F04D10C4B3C
:102120001B6813F0020F06D102214FF4827004F0F5
:10213000E0FA28B908BD0021044804F061FBF3E788
:102140000121024804F05CFBF4E700BF5C000020C2
:102150009427002008B50A4BBFF35B8F53E8002F8C
:1021600022F0020143E800100028F7D1BFF35B8F93
:1021700012F0010F00D008BDFFF740FFFBE700BFE2
:102180009427002070B5064600220121104600F079
:1021900043FA002000F030FA4FF080430122C3F8E8
:1021A000182504F0C0FA0024012C12D8214630462C
:1021B00004F0BFFA05462146304604F0C7FA064946
:1021C00003F0A7FF002805DB0123AB601C44E4B249
:1021D000EAE7002070BD00BF3896000010B5044645
:1021E000124B0121BFF35B8F53E8002F43E800102F
:1021F0000028F9D1BFF35B8F3AB1012C11D0022C2A
:1022000002D1012004F05BFB10BD094804F09EFAE6
:10221000084900234B60CB6001238B6003F095FFDE
:10222000EBE7002004F04BFBEEE700BF982700200F
:102230005C0000203427002020F07F40014BC3F8D1
:102240004005704700100140014BD3F8400570472E
:102250000010014082B0044B00221A601B680193F9
:10226000019B02B0704700BF40110140024B4FF488
:102270008032C3F84423704700100140024B4FF4F2
:102280008032C3F80823704700100140024B4FF41E
:102290008032C3F80423704700100140014BD3F88B
:1022A000040570470010014038B5FFF7D3FFFFF772
:1022B000CBFF054D2C68214604F011FB04442C6033
:1022C00002F0BEFE38BD00BF9C27002038B5FFF7E6
:1022D000E5FF0446FFF7B8FF0546FFF7BBFF2046C2
:1022E000FFF7AAFFFFF7C2FF2146284604F0F7FADE
:1022F000012805D0054B4FF40032C3F8802138BDCA
:102300000F2006F0A1FCFFF7A5FFF3E700E100E0D6
:1023100038B50F4D0024C5F80845FFF79BFF0D4B5E
:102320004FF40032C3F88021FFF7B0FF22460121AD
:10233000112000F071F9112000F05EF90123064A26
:1023400013602B602046FFF749FF204638BD00BFD1
:102350000010014000E100E00810014038B5B0F184
:10236000FF3F1ED0441E114B9C4201DC002C1BDDA4
:102370000E4B9C4200DD0E4CFFF790FF0D4B1D688D
:10238000294604F0ACFAB0F5000F00D30024204435
:102390000130B0F5000F00D30548284404F0D5FA09
:1023A00038BD00F50000DDE70024E5E7FEFF7F0013
:1023B000FFFF7F009C27002010B54FF02003EFF3B4
:1023C000118483F31188BFF36F8FFFF767FF044B0E
:1023D000196804F084FA84F31188BFF36F8F10BD7D
:1023E0009C27002038B54FF02003EFF3118583F3CD
:1023F0001188BFF36F8FFFF751FF054B1C68214613
:1024000004F06DFA204485F31188BFF36F8F38BD57
:102410009C27002010B5114C032323616361104AEF
:10242000A261104BE3614FF4806323620023A36237
:102430006362E36222660C4A62661022A266236728
:10244000E36663670949E01D04F0FFFA0849204686
:1024500004F0FBFA2023A37110BD00BFA0270020C9
:102460005096000058280020482800205C96000064
:10247000609600002DE9F84304460E46154600EB31
:1024800040032D4A02EBC302936A576ABB424BD802
:1024900000EB4002284901EBC202D2F82080A8EBF1
:1024A000070909F1FF32954204D913449D4216D918
:1024B00000203EE0DFF88080631C03EB430308EB61
:1024C000C30358682A463146384404F0E8FA3D44CC
:1024D00004EB440408EBC4046562012029E0431CBA
:1024E00003EB4303144A02EBC30358684A463146E0
:1024F000384404F0D4FAA7EB08077F1907D104EB9E
:1025000044040D4B03EBC4046762012011E0631C1B
:1025100003EB4303084A02EBC3033A4606EB090107
:10252000586804F0BCFAEAE7DB1B013BAB42C1D2BE
:102530000020BDE8F88300BFA0270020064B00EB79
:10254000400203EBC202926A00EB400003EBC000C2
:10255000406A801A704700BFA0270020094A93688C
:10256000986709490968D96708494B6843F080535F
:102570004B60002383F31188BFF36F8F9368D86F8C
:10258000704700BFDC2C00202499000000ED00E023
:102590000F498A684FF038001044EFF3098C80E847
:1025A000F01F202080F31188BFF36F8F094F4FF089
:1025B0000066CA698A603E60906F0023936780F36B
:1025C000118802F1380090E8F01F8CF309887047F9
:1025D000DC2C002004ED00E01EF0040F0CBFEFF334
:1025E0000880EFF30980816911F8021C0229FFD0ED
:1025F00001B504F0CDF901BD43B2002B08DB00F0BA
:102600001F005B09012202FA00F0024A42F823008F
:10261000704700BF00E100E0013143B2002B08DB4E
:102620004901C9B203F1604303F5614383F8001324
:10263000704700F00F004901C9B2014B19547047AF
:1026400014ED00E080B504460F4616461D4604F022
:1026500097F9384631462A46044B202583F30988EA
:10266000A04785F31188BFF36F8FFEE71855002050
:10267000014910220A60704710ED00E030BFFFF7FB
:10268000FDBF00BF08B50E4B0E4A22F07F029A60D4
:10269000BFF34F8FBFF36F8FD3F8882022F47002FF
:1026A000C3F88820EFF3148323F0040383F3148822
:1026B00002F082FA02F08CFA00F022F902F0C4FA79
:1026C00000ED00E00000000001B5EFF30580A0F18F
:1026D00010004FEAC0000449014409C99847BDE809
:1026E0000140024908470000688D0000FD280000F5
:1026F00004F019FA202080F3118808484FF4006193
:10270000401880F30988EFF314800221084380F316
:102710001488BFF36F8FFFF7B5FF00001855002036
:10272000EFF30880EFF30981724601B500F094F8E9
:1027300001BD00BF10B514460F4B9A6A9A6A9B6A96
:1027400013F0020F0BD00C4B5A6B9B6A13F0800FE7
:1027500005D021B1084A936A23F080039362064BA7
:102760009A6A9A6A9A6A9A6A42F0FF029A6204F036
:102770001BF92070002010BD00ED00E010B51446DC
:10278000124B9A6A9A6A9B6A13F4007F0BD00F4B24
:102790009A6B9B6A13F4004F05D021B10B4A936AE0
:1027A00023F400439362094B9A6A9B6A13F4807F77
:1027B00001D1064B9B6A054A936A43F47F439362B7
:1027C00004F0F2F82070002010BD00BF00ED00E022
:1027D000074B9A6A9A6A9A6A9A6A9A6A9A6A9A6A8B
:1027E0006FEA02426FEA12429A620020704700BF0D
:1027F00000ED00E000230B70144BDA6A12F00202C5
:1028000021D110B50446D86A10F0804010D028338A
:102810001B7843B90E4B1B785BB90E4B1B889BB2E0
:102820006BB9104604E00A4601212046FFF782FFFB
:1028300010BD0A4601212046FFF7A0FFF8E7204619
:10284000FFF7C6FFF4E70020704700BF00ED00E08F
:1028500029ED00E02AED00E070B58AB00C46224B6D
:102860005968C1F30801002383F31188BFF36F8F08
:1028700002F07F43B3F17F4F15D102F00C03082B18
:1028800014D012F0080F0BD000260DF127022046BD
:1028900004F08CF805469DF8273053B10AB070BD9E
:1028A00004460126F1E700263446EEE700263446CA
:1028B000EBE72022214601A804F0F1F84EB1089B75
:1028C000C3F308025AB96FEA53236FEA432308930C
:1028D00005E0089B23F4FF7323F00103089301A98B
:1028E000284604F051F8D9E700ED00E0024A5369A8
:1028F00043F010035361704700ED00E0704700BFE4
:10290000002206E002F00F01094B0B44202119764A
:1029100001322F2A0ADC53B2002BF3DB03F16043B0
:1029200003F56143202183F80013F1E7704700BFEE
:10293000FCEC00E038B504464FF02003EFF31185BE
:1029400083F31188BFF36F8F02F094FA0A4B9B68F0
:10295000A34203D0284606F00BF938BD074B5B684D
:10296000C3F308032BB1054A536843F08053536007
:10297000F0E72846FFF7F2FDDC2C002000ED00E038
:1029800000B585B0084B0193084B0293084B0393A5
:1029900001AB0093074B084A0121684604F051F847
:1029A00005B05DF804FB00BF00000020000000003F
:1029B00000000B060000042000000020064A906082
:1029C0000B6823F01F03034343F01003D3608B68AD
:1029D00043F001031361704790ED00E010B5072844
:1029E00004D80446FFF7EAFF204610BD4FF000046C
:1029F000012363F302046FF3C504074B074A9B1AD4
:102A0000C3F3C90363F38F1402460549204603F05C
:102A1000F1FC6FF01504E7E7F88E0000E88E000087
:102A20006C9600002DE9F84380460F4699461446FF
:102A3000002509E03146E0B203F0E4FF044610F15E
:102A4000160F22D001340135BD421EDA58F8256038
:102A50007368002BF7D0B9F1000FEBD0304603F0CC
:102A6000C0FF0028E6D1012363F302006FF3C50025
:102A7000074B084A9B1AC3F3C90363F38F102A4616
:102A8000054903F0B7FC6FF015042046BDE8F88354
:102A9000F88E0000E88E00009496000010B5034CFC
:102AA00001232278FFF7BEFF207010BD0D2D0020FE
:102AB000034B05225A60BFF34F8FBFF36F8F7047F0
:102AC00090ED00E0BFF35F8F014B00225A6070472A
:102AD00090ED00E038B50E4B1D68082D15D8FFF7B6
:102AE000F1FF0024A5420AD9094B596804EB4402BE
:102AF000930019442046FFF761FF0134F2E7054BCC
:102B00001D70FFF7D5FF002038BD4FF0FF30FBE709
:102B1000C89600000D2D0020014B1860704700BFC3
:102B2000100000204FF02003EFF3118283F311888F
:102B3000BFF36F8F01230649C1F840354FF0804144
:102B4000C1F8783582F31188BFF36F8F002070478A
:102B500000E0014030B108B58001034B43F00103B0
:102B6000984708BD704700BF508F0000F0B443681D
:102B70005F68374B1340374CA34227D012D8062B3F
:102B800026D004D9B3F5801F09D1012416E00BB378
:102B9000022B01D1042411E06FF0150053E06FF017
:102BA000150050E02C4CA34216D0B3F5A00F01D174
:102BB000032403E0B3F5800F47D1022412F0100F75
:102BC0000CD112F0200F27D0012508E00724F5E7EB
:102BD0000624F3E70024F1E70524EFE70325C2F319
:102BE000402312F4807F0CBF0126002612F4007FE0
:102BF00006D012F4006F11D001228A40C7F80825D0
:102C00004268127A01F01F0141EA42111F290DD9D1
:102C100001F01F01114A0BE00025E0E712F4806F7C
:102C2000EED001228A40C7F80C25E9E74FF0A04218
:102C300043EA460343EA850343EA042301F5E071CE
:102C400042F821300020F0BC70476FF01500FAE721
:102C50000600F000060010000200400000030050D3
:102C6000F0B4C6684768F1687269B369134321EA32
:102C700003010122002012E04FF0020C1EE04FF091
:102C8000A04503F5E07355F8234024F4403444EAAA
:102C90000C4445F8234021EA02010130520099B169
:102CA0000A42FAD03C7A00F01F0343EA4413346925
:102CB000C44014F0010FDFD14FF0030C1F2BDED9FD
:102CC00003F01F03014DDCE7F0BC70470003005028
:102CD000F0B4C3684768D9685A699869024321EA21
:102CE00002017A68D2F810251869504021EA0000E4
:102CF000012200240DE04FF0A04603F5E07356F8E2
:102D0000235025F4403546F8235021EA02010134CE
:102D1000520061B11142FAD03D7A04F01F0343EA38
:102D200045131F2BE7D903F01F03024EE5E7F0BC64
:102D3000704700BF0003005030B4194BD3F8045360
:102D4000EDB2002300E00133072B26D803F5A27271
:102D5000134C54F82220C2F305229142F3D125FAF4
:102D600003F212F0010FEED001229A40D143BFF3DB
:102D70005B8F50E8004F0C4040E80045002DF8D133
:102D8000BFF35B8F064903F5A27351F8230020F0CF
:102D9000010041F82300C1F8082330BC704700BF90
:102DA000006000400023072B4AD870B483B0012490
:102DB0009C40BFF35B8F50E8005F45EA040640E8A3
:102DC000006CBCF1000FF6D1BFF35B8FDD4015F056
:102DD000010F08D00133DBB2072BE8D96FF01200E6
:102DE00003B070BC704703F14000800080B2164D04
:102DF00003F5A27355F8236026F44F3626F4407687
:102E000045F8236055F82360090201F47C5112044F
:102E100002F440320A43324345F8232000F1804255
:102E200002F5C0420020106012680192019A55F824
:102E3000232042F0010245F82320C5F80443CFE7E0
:102E40006FF01200704700BF0060004070B50D4683
:102E5000C66843681B7A01F01F0444EA4314214604
:102E60002448FFF769FF1F2C21D904F01F00224AD4
:102E700000F5E07152F8213023F4403342F821305C
:102E8000F368EB4013F0010F32D07369EB4013F09D
:102E9000010F18D0B369EB4013F0010F0BD131696A
:102EA00021FA05F515F0010F0BD0012204E02046B0
:102EB0004FF0A042DCE7032221460E48FFF772FFE5
:102EC00017E00222F8E7316921FA05F515F0010F44
:102ED0000CD1032100F5E07052F8203023F4403388
:102EE00043EA014342F82030002002E00221F1E7EA
:102EF000002070BD902C00200003005070B5C46805
:102F000045682E7A01F01F0545EA4615B2F5A03F47
:102F100025D0B2F5005F34D0E56801268E403543F8
:102F2000E560B2F5A03F32D0626901258D4022EA0A
:102F300005026261B3F5C02F2ED0A26901258D4034
:102F400022EA0502A261B3F5802F2AD0236901226B
:102F50008A4023EA02032361FFF778FF70BD1F2D2B
:102F60000CD905F01F05114E05F5E07556F82550F2
:102F700015F0010FCDD06FF02200EFE74FF0A04623
:102F8000F2E7E56801268E4025EA0605C8E7626992
:102F900001258D402A43CCE7A26901258D402A43B3
:102FA000D0E7236901228A401343D4E7000300508D
:102FB00008B50B4B1B780BB1002008BD084B012254
:102FC0001A70002205210620FFF726FB0620FFF7D6
:102FD00013FB044B4FF00042C3F80423ECE700BF9F
:102FE0000E2D00200060004070B584B000230293D5
:102FF0000393484B1C680CB9002111E0464D28464C
:10300000FFF766FE029005F11000FFF761FE0390E6
:10301000404B00221A601B680093009BECE70131D3
:1030200007292FD801F140039B009AB201238B405E
:103030003A48D0F804030342F1D002F1804303F58B
:10304000C0431B68002BEAD001F5A273334850F847
:103050002300C0F34033C0F30420012505FA00F03B
:1030600004AD05EB830353F8085C054343F8085CA3
:1030700002F1804303F5C04300221A601B680193EC
:10308000019BCCE7029E2EB9039EF6B9002C37D1E6
:1030900004B070BD204BDB68596819B10D4649B1C9
:1030A0000D6807E00D4605E06DB12B4605B12B68B4
:1030B00029461D460029E7D08A683240F4D04B6883
:1030C00015489847F0E72B46F2E7134BDB69596840
:1030D00019B10D4649B10D6807E00D4605E06DB127
:1030E0002B4605B12B6829461D460029CED08A689B
:1030F0003240F4D04B680A489847F0E72B46F2E795
:10310000054C2046FFF7ACFD04F11000FFF7A8FDC9
:10311000BEE700BF7C6100409C00002000600040D2
:10312000AC000020034BD3F8003413F0010FF9D0AA
:10313000704700BF00E00140024B0B6001231360A9
:10314000704700BF942C0020004870475097000043
:1031500010B504F019F8034C206004F011F8606019
:10316000002010BD942C0020054B1B6823B9054B93
:103170001B781BB101207047012070470020704769
:103180001C210040102D002082B0054A002313604E
:1031900012680192019A034A137002B0704700BF8F
:1031A0001C210040102D0020B1F5164F6DD03BD8EA
:1031B000B1F5165F6BD00AD9B1F5E14F72D025D9C0
:1031C00047F6122399422CD14FF4000313E0B1F5D6
:1031D000966F5ED007D9B1F5166F60D0B1F5965FE6
:1031E00011D13A4B07E0B1F5967F55D0B1F5167F76
:1031F00006D14FF41C33364AC2F8243500207047FC
:103200006FF0150070476FF015007047B1F5615F02
:103210004AD0B1F5964F01D12E4BECE76FF0150077
:1032200070476FF015007047B1F5613F3FD009D985
:10323000B1F5612F42D01DD9274B994243D14FF0B0
:103240008053D8E7B1F5963F33D004D9B1F5E13FCB
:103250000DD1224BCFE74DF6C02399422BD0B1F5CB
:10326000614F01D11E4BC6E76FF0150070476FF03C
:10327000150070471B4B994222D0B1F5E12F01D1C7
:10328000194BB8E76FF015007047184BB3E7184BB0
:10329000B1E74FF49E23AEE74FF4A033ABE74FF412
:1032A0001D23A8E7134BA6E74FF46C13A3E7124BBB
:1032B000A1E7124B9FE74FF465039CE7104B9AE799
:1032C0004FF0806397E76FF01500704700B0130070
:1032D0000020004000A04E0040420F0000E0D70157
:1032E00000F0EB0090D0030000705F0700509D00DD
:1032F0000050270000F0750000B0AF0300903A01C5
:1033000000D0BE0E094B1B6863B182B0074B002092
:1033100018601B680193019B054BD3F818350B709F
:1033200002B070474FF0FF30704700BF08210040E7
:1033300000200040024BD3F88004C3F8800470479B
:103340000020004030B583B005460C464B79012B78
:1033500006D0032B11D06FF02203184603B030BD06
:1033600000238DF80630A379032B36D1E37943B1DE
:10337000012B10D06FF02203EFE710238DF80630F9
:10338000F1E700238DF80430237943B1022B20D0DC
:103390006FF02203E1E701238DF80430F4E7002306
:1033A0008DF8053021682846FFF7FEFE0346B8B9C0
:1033B0009DF805109DF806009DF8042001430A437E
:1033C0000949C1F86C25EA6894E8030082E8030023
:1033D000C3E70E238DF80530E4E76FF02203BCE766
:1033E0006FF02203B9E700BF00200040F8B50E4699
:1033F0001546002427462B1B002B0BDDFFF7B4FEE0
:1034000040B1FFF7C1FE631C345D0348C0F81C45A2
:10341000DCB2EFE73846F8BD0020004010B483B0BE
:1034200000231846D41A002C0FDD094C246864B11F
:10343000074800240460006801900198581C054C5E
:10344000D4F81845CC54C3B2EBE703B010BC7047B6
:103450000821004000200040014B01221A707047F3
:103460000F2D0020024B0422C3F80423704700BF35
:1034700000200040024B0422C3F80823704700BF1D
:103480000020004008B50A4BD3F8043313F0800F36
:1034900009D0084B1B780BB1002005E0FFF764FE54
:1034A00018B1012000E0002008BD0020FCE700BFAB
:1034B000002000400F2D0020024B1868003818BF74
:1034C0000120704708210040024B4FF40072C3F8FE
:1034D0000423704700200040024B4FF40072C3F8F1
:1034E000082370470020004010B504460D4BD3F868
:1034F000043313F0800F07D10A4BD3F8043313F0D1
:10350000040F07D1002010BDFFF7BCFF0028F3D047
:103510000120F8E72046FFF7CFFF0028F3D0012075
:10352000F1E700BF00200040024B1960024B1A6017
:10353000704700BF9C2C0020A02C002008B5104B29
:1035400000221A7005F0C3FA0E4B01221A60083BE4
:103550008022C3F804234FF02002EFF3118382F39B
:103560001188BFF36F8F084A12781AB1074A0421F5
:10357000C2F8001183F31188BFF36F8F08BD00BF3D
:103580000F2D002008200040102D002000E100E059
:1035900038B50C4605F052FBC0B96425194B012221
:1035A000BFF35B8F53E8001F002903D143E80020DD
:1035B0000028F7D1BFF35B8F0BD02120002101F051
:1035C000C9FC013D15F0FF05E8D102E00D4B0122D9
:1035D0001A60FFF7D9FD0C4B01221A60083BC3F8B3
:1035E0001C454FF47A74FFF7BFFD20B9012003F0AA
:1035F00096FD013CF7D1054B01221A60014B0022D8
:103600001A6038BDA42C0020082000400C20004087
:1036100030B583B01E4A0021C2F800154FF0A04318
:103620004024C3F808450324C3F81847C3F82017FB
:103630000825C2F814550625C2F80C552025C3F8F4
:103640000855C3F81447C3F81C170523C2F80835FA
:103650000723C2F81035C168FFF774FE044610B1A5
:10366000204603B030BD0A4B0422C3F800250949A7
:1036700000220A6009680191019901211960064B35
:1036800019700220FEF7C8FF0220FEF7B5FFE7E73A
:103690000020004008210040102D002000B583B01C
:1036A000124B1B7813B1124B1B688BB9114B1B6863
:1036B0002BB1104B00221A601B680193019B0E4B2B
:1036C0001B6813B10D4A1168984703B05DF804FBFD
:1036D0000B4B8022C3F808230C3301221A6005F03B
:1036E000F7F9024B00221A70EFE700BF0F2D002000
:1036F0001C210040242100409C2C0020A02C0020F4
:103700000020004043681A68B1F5164F6FD03AD8D0
:10371000B1F5165F6ED00AD9B1F5E14F75D024D955
:1037200047F6122399422BD14FF4000313E0B1F571
:10373000966F61D007D9B1F5166F63D0B1F5965F7A
:1037400010D13C4B07E0B1F5967F58D0B1F5167F0C
:1037500005D14FF41C33C2F82435002070476FF0B8
:10376000150070476FF015007047B1F5615F4ED0DE
:10377000B1F5964F01D1304BEDE76FF01500704772
:103780006FF015007047B1F5613F42D009D9B1F52E
:10379000612F46D01FD9294B994248D14FF0805311
:1037A000D9E7B1F5963F37D005D9B1F5E13F0FD153
:1037B0004FF0EB73CFE74DF6C02399422ED0B1F511
:1037C000614F02D14FF46B03C5E76FF015007047EE
:1037D0006FF0150070471A4B994225D0B1F5E12FD3
:1037E00002D14FF0E863B6E76FF0150070474FF471
:1037F0001D03B0E7134BAEE74FF49E23ABE74FF446
:10380000A033A8E74FF41D23A5E70F4BA3E70F4B09
:10381000A1E74FF06C739EE70D4B9CE74FF46503F7
:1038200099E74FF0706396E74FF0806393E76FF08E
:103830001500704700B0130000A04E0040420F007A
:1038400090D003000050270000C0750000F03A003F
:1038500000903A01F0B583B00C46164643681D68E7
:10386000C7680023C5F800350A681F2A1BD902F073
:103870001F02454901239340C1F8083523681F2BD7
:1038800014D903F01F03404A03F5E073032142F803
:1038900023106368B3F1FF3F12D01F2B09D903F047
:1038A0001F03394A07E04FF0A041E3E74FF0A04281
:1038B000EAE74FF0A04203F5E073002142F823103D
:1038C00022686368C5F80C25C5F81435A368B3F100
:1038D000FF3F0CD01F2B03D903F01F032A4A01E03E
:1038E0004FF0A04203F5E073002142F82310E36893
:1038F000B3F1FF3F1AD01F2B03D903F01F03224956
:1039000001E04FF0A041012202FA03F3C1F80835AB
:10391000E3681F2B03D903F01F031B4A01E04FF09C
:10392000A04203F5E073032142F82310E268A36884
:10393000C5F80825C5F81035C16803F07FFA00BB4B
:103940000823C5F800356368B3F1FF3F0ED00023AC
:10395000C5F81031D5F810310193019B07F1100320
:10396000C5F834350123C5F838352B604EB1BB6836
:103970009B68C5F844350023C5F848350123AB6082
:10398000EB6003B0F0BD00BF0003005030B585B060
:1039900005460A4B6C460FCB84E80F00002201213C
:1039A0002820FEF739FE2820FEF726FE01222146B8
:1039B0002846FFF74FFF05B030BD00BF408F000025
:1039C0000D4B1A68B2F1FF3F05D00C4B1B68082A5B
:1039D00008D0002070470A4B1A7808331B68C3F3DD
:1039E0000313F4E7032B03D8DFE803F00404040413
:1039F0000020704701207047300100103401001092
:103A0000E00F00F00D4B1A68B2F1FF3F05D00C4BF0
:103A10001B68082A08D0002070470A4B1A78083320
:103A20001B68C3F30313F4E7032B03D8DFE803F0A9
:103A30000404040400207047012070473001001086
:103A400034010010E00F00F0064B1B68064A1268B4
:103A5000082B01D0002070470AB1002070470120D8
:103A6000704700BF3001001034010010064B1B6886
:103A7000064A1268082B01D0002070470AB10020C6
:103A800070470120704700BF300100103401001062
:103A9000064B1B68064A1268082B01D000207047AD
:103AA0000AB1002070470120704700BF30010010AC
:103AB00034010010064B1B68064A1268082B01D01F
:103AC000002070470AB1002070470120704700BFF6
:103AD00030010010340100100D4B1A68B2F1FF3FA5
:103AE00005D00C4B1B68082A08D0002070470A4BF1
:103AF0001A7808331B68C3F30313F4E7032B03D8C6
:103B0000DFE803F00404040400207047012070473C
:103B10003001001034010010E00F00F0014B024AA8
:103B20001A607047400000200090D00308B5FFF7EE
:103B300047FF40B14FF080430022C3F80C21C3F887
:103B40001021C3F83825FFF75DFF002846D04FF05D
:103B50008052D2F804145B4BC3F82015D2F8081435
:103B6000C3F82415D2F80C14C3F82815D2F8101491
:103B7000C3F82C15D2F81414C3F83015D2F8181461
:103B8000C3F83415D2F81C14C3F84015D2F8201429
:103B9000C3F84415D2F82414C3F84815D2F82814F1
:103BA000C3F84C15D2F82C14C3F85015D2F83014C1
:103BB000C3F85415D2F83414C3F86015D2F8381489
:103BC000C3F86415D2F83C14C3F86815D2F8401451
:103BD000C3F86C15D2F84424C3F87025FFF734FFFE
:103BE00010B1394B394A1A60FFF740FF18B1384B12
:103BF000FB22C3F81825FFF74BFF48B135490B6886
:103C000023F00F03344A126802F00F0213430B60D3
:103C1000FFF750FF18B1314B4FF400721A60FFF7F5
:103C20005BFF60B14FF08043D3F8003413F0010F15
:103C300005D04FF080436FF00102C3F800244FF02D
:103C40001023D3F80032002B08DB4FF01023D3F8F9
:103C50000432002B02DBFFF761FF08BD204B01227D
:103C6000C3F804251E4BD3F80034002BFAD04FF0D4
:103C700010231222C3F80022194BD3F80034002B72
:103C8000FAD04FF010231222C3F80422144BD3F8B9
:103C90000034002BFAD0124B0022C3F80425104B3D
:103CA000D3F80034002BFAD0BFF34F8F0D49CA6808
:103CB00002F4E0620C4B1343CB60BFF34F8F00BFA5
:103CC000FDE700BF00C000408C5600404881030063
:103CD00000F00040E40E0040580200104096024000
:103CE00000E0014000ED00E00400FA05024B002274
:103CF000C3F80425704700BF00E00140024B0122D9
:103D0000C3F80425704700BF00E00140024B0222C7
:103D1000C3F80425704700BF00E00140044BD3F80E
:103D2000003413F0010FF9D00160BFF35F8F7047CB
:103D300000E0014010B5044603F006FA08B908484F
:103D400010BDFFF7E3FF074BC3F80845054BD3F859
:103D5000003413F0010FF9D0FFF7C8FF0248EFE776
:103D60000A00AD0B00E001400000AD0B0268124BF1
:103D70009A4215D1C269A3F11023A3F1EF139A421D
:103D800010D18368012B0FD8C36813B10269934225
:103D90000CD0436963B1826993420BD00020704715
:103DA00001207047012070470120704701207047B3
:103DB000002070470120704755AA00FF70B5114BD5
:103DC0009D68B5B12846FFF7D1FF064698B9EB6864
:103DD00013B10126304670BD2C69002CFAD0204664
:103DE000FFF7C4FF48B9E368AB4208D12546246910
:103DF000F3E70126EEE70126ECE70126EAE70126D4
:103E0000E8E700BFC82C0020002800F0928038B5F9
:103E10000546484B1B68002B6CD0464A9268002A26
:103E200068D0834204D8434A52681344834203D87B
:103E3000414B1B6801209847A5F120042046FFF75D
:103E400095FF18B13C4B1B680120984755F8183C6A
:103E5000012B03D0384B1B6801209847002345F8FD
:103E6000183C55F8143CCBB19A68002A43D155F858
:103E70001C2C59680A4420325A6055F8143C55F8F5
:103E8000102C1A6155F8145C2B6903B1DD602022F7
:103E90000021204602F027FE23462C4625691DB34B
:103EA000AA680ABB6B6862681344203363602B699D
:103EB000236163690BB323B3A2699A61A3690BB150
:103EC00062695A616B696361AA69A261EBB19C6125
:103ED000A36903B15C61236903B1DC602022002186
:103EE000284602F000FE2B4693B1124B1B6913F0DB
:103EF000020F15D138BD0023D0E7A269002ADAD11C
:103F0000E0E7A2690B4BDA60D8E70A4BDC60DFE739
:103F1000084BDB68A36103B15C61064BDC60E4E73E
:103F2000FFF74CFF0028E5D0034B1B6801209847A2
:103F3000E0E77047C82C00204800002070B54F4BC8
:103F4000DC681D68002D5AD09D68002D57D001FBFC
:103F500000F6002800F08880002900F08780B6FB7A
:103F6000F0F0884240F0848016F1040F00F2828065
:103F700016F0030F08D026F00305043534B163684A
:103F8000AB4203D2A469F9E73546F7E7002C73D0BA
:103F9000A3681BB13A4B1B68012098476268521B0B
:103FA000232A2ED905F120016318203A5A600022F5
:103FB0009A60DC6022691A61324860503249D961E6
:103FC00002B1D36062695A61A1699961002A3FD048
:103FD00093619A6902B153610122A2606560236115
:103FE00000236361A361254B1B6913F0010F32D1DC
:103FF00004F1200532460021284602F074FD2846CF
:1040000070BD0123A3606369ABB1A2699A61A36922
:104010000BB162695A6100236361A361174B1B698D
:1040200013F0010F0BD104F1200532460021284680
:1040300002F059FDE3E7A269104BDA60E7E7FFF70A
:10404000BDFE0028EFD00E4B1B6801209847EAE721
:104050000A4AD360BDE7FFF7B1FE0028C8D0084B7D
:104060001B6801209847C3E70025C8E70025C6E77D
:104070000025C4E70025C2E72546C0E7C82C00207C
:104080004800002055AA00FF669911EE38B5054694
:104090000C4614220021134802F025FD1249134852
:1040A00000F038F8232C1CD915F0030304D01C446D
:1040B000043CC3F104031D4422460021284602F0BB
:1040C00012FD084B1D605C609D60203C6C609A682E
:1040D000074911609A68A1F11021A1F1EF11D16196
:1040E000DA6038BDC82C0020093E00003D3F0000CA
:1040F00055AA00FF08B5024B1B68984708BD00BFD2
:104100004400002008B5024B1B68984708BD00BF5B
:104110004C000020024B1860024B196000207047D1
:10412000440000204C00002031B108B50A46034B82
:104130001B680021984708BD704700BF5000002051
:10414000F8B504460D46476800F10806304603F00E
:10415000A2FB874251D16368B3F5807F4FD800211D
:10416000304603F098FD00282ADD0021304603F098
:104170006AFB28B3CDB104F12C060021304603F0D0
:104180008AFD00281EDD0021304603F05CFBC8B12B
:1041900004F138060021304603F07DFD002811DDD2
:1041A0000021304603F04FFB60B1002104F1140000
:1041B00003F071FD002824DD35B9ADB92846F8BDFE
:1041C000124DFBE7114DF9E7002104F1440003F023
:1041D00062FD002806DD002104F1500003F05BFDC4
:1041E0000028EADC094DE9E7002104F15C0003F056
:1041F00052FD002807DD0025E0E7044DDEE7034D12
:10420000DCE7024DDAE7014DD8E700BF80BFFFFFD2
:1042100070B5044600221146FFF792FFE0B906464A
:1042200004F10805284603F01FFB7F2816D9143433
:104230000021204603F007FB60B1204603F014FB89
:10424000012807D92946204603F0DDFC002801DAC1
:10425000304670BD024EFBE7014EF9E7004EF7E72E
:1042600000BEFFFFF0B587B004460D46164600229B
:104270001146FFF765FF98BB03A803F053FA626885
:10428000294603A803F00DFB054630B103A803F04F
:104290004FFA15BB284607B0F0BD04F108052946C2
:1042A00003A803F0B0FC002802DB6FF00305EDE784
:1042B000676804F1680300932B4604F1140203A914
:1042C000084604F04BF805460028DFD13A4631464F
:1042D00003A803F015FB0546D8E7A5F58545D9E702
:1042E000004DD7E780BFFFFF0023036043600B460C
:1042F000B9B9194A8260194AC260194A0261194A59
:104300004261194A8261194AC261194A026202F184
:104310007452A2F52302A2F6924242628366002002
:104320007047144A8260144AC26002F1794202F571
:10433000740202F501620261104A4261104A826110
:1043400002F1D14202F5C01202F51E62C2610D4AAD
:1043500002620D4A4262E1E767E6096A85AE67BB21
:1043600072F36E3C3AF54FA57F520E518C68059B57
:10437000ABD9831FD89E05C107D57C3639590EF7B6
:10438000310BC0FFA78FF964A44FFABE2DE9F04F9F
:10439000D1B00790002306E09A1C50F8222008AC08
:1043A00044F823200133072BF6D900220F2A11D815
:1043B00011F8224001EB820043781B0443EA0463B6
:1043C000847843EA0423C078034310A840F82230DD
:1043D0000132EBE74FF0000E42E10F9B0C9E4FEADB
:1043E000F62181EAB61181EA766119440E9C0D9896
:1043F00084EA0003334063401944DFF8348758F8F7
:104400002E3019440DF1400C5CF82E301944089DF3
:104410004FEA753A8AEAB50A8AEAB55A099F05EA67
:1044200007030A9A45EA070902EA090943EA090368
:104430009A440B9B01EB030951444FEAF92383EAA9
:10444000B91383EA79631C4486EA000309EA03038B
:1044500043401C440EF1010A58F82A301C445CF811
:104460002A301C444FEA713383EAB10383EAB15323
:1044700005EA010A45EA010B07EA0B0B4AEA0B0AB7
:10448000534422441C444FEAF22383EAB21383EAE2
:104490007263184486EA09031340734018440EF10E
:1044A000020A58F82A3018445CF82A3018444FEAB7
:1044B000743383EAB40383EAB45301EA040A41EA99
:1044C000040B05EA0B0B4AEA0B0A53440744184451
:1044D0004FEAF72383EAB71383EA77631E4489EA36
:1044E00002033B4089EA03031E440EF1030A58F815
:1044F0002A301E445CF82A301E444FEA703383EAA7
:10450000B00383EAB05304EA000A44EA000B01EA6C
:104510000B0B4AEA0B0A534435441E444FEAF52379
:1045200083EAB51383EA7563994482EA07032B4053
:10453000534099440EF1040A58F82A304B445CF871
:104540002A904B444FEA763989EAB60989EAB65986
:1045500000EA060A40EA060B04EA0B0B4AEA0B0AD9
:10456000D14419440F914B440B934FEAF12989EA46
:10457000B11989EA71694A4487EA050901EA09091A
:1045800087EA090991440EF1050A58F82A204A449D
:104590005CF82A904A444FEA733A8AEAB30A8AEAF4
:1045A000B35A06EA030946EA030B00EA0B0B49EA91
:1045B0000B09CA4404EB0209CDF8389052440A9220
:1045C0004FEAF92484EAB91484EA7964274485EA35
:1045D000010409EA04046C403C440EF1060A58F850
:1045E0002A703C445CF82A703C444FEA723787EAF0
:1045F000B20787EAB25703EA020A43EA020B06EA65
:104600000B0B4AEA0B0A574420440D903C44099492
:104610004FEAF02787EAB01787EA70673D4481EADE
:10462000090900EA090981EA090129440EF1070094
:1046300058F8205029445CF8200001444FEA7430B7
:1046400080EAB40080EAB45002EA04052243134031
:104650002B4303440E440C960B4408930EF1080EB2
:10466000BEF10F0F7FF6B9AE10263F2E00F24D823D
:104670000F9A0C9B4FEAF32787EAB31787EA736711
:104680003A440E980D9D80EA05071F4047403A4482
:10469000DFF89CB45BF826701744B31E1A4610ABC3
:1046A000049253F822204FEAF24484EA724484EAE6
:1046B0009224F21F53F822201444A6F10F0A53F853
:1046C0002AC04FEABC4282EAFC1282EADC021444AD
:1046D000A6F1100253F82220224443F826203A443F
:1046E00008994FEA713C8CEAB10C8CEAB15E099FE3
:1046F0003C460C400A990091089941EA070C009940
:1047000001EA0C0C44EA0C0CF4440B9C1444624483
:104710004FEAF42888EAB41888EA746880440C994F
:1047200081EA050904EA090985EA0909C844711CF6
:104730005BF821008044701E059053F820004FEA7A
:10474000F04C8CEA704C8CEA902CB01F53F820008F
:104750008444A6F10E0E53F82E904FEAB94080EA39
:10476000F91080EAD900604453F82A904844029135
:1047700043F8210008EB00094FEA723888EAB208D2
:1047800088EAB258089901EA020041EA020C01974E
:1047900007EA0C0C40EA0C0CC444009800EB090832
:1047A000E1444FEAF82080EAB81080EA78600544D6
:1047B0000C9981EA040008EA000048400544B01C56
:1047C00001465BF82000054453F826004FEAF04C00
:1047D0008CEA704C8CEA902C701F53F820008444B3
:1047E000A6F10D0A53F82A004FEAB04053F82A7098
:1047F00080EAF71080EAD700604453F82EC0604486
:10480000039143F8210005444FEA793C8CEAB90C46
:104810008CEAB95C02EA090042EA090E089901EA49
:104820000E0E40EA0E008444019F07EB050E05EBD7
:104830000C0700974FEAFE2080EABE1080EA7E60F7
:104840000C990D1884EA08010EEA0101614068180C
:10485000F71C5BF827100144029D53F825004FEA2E
:10486000F04585EA704585EA9025301F53F8200011
:1048700005440195A6F10C0C53F82C004FEAB0400A
:1048800053F82C5080EAF51080EAD500019D2844A9
:1048900053F82A502844069743F82700014400980B
:1048A0004FEA7035074685EAB00585EAB05509EA52
:1048B000000049EA070A02EA0A0A40EA0A00054437
:1048C000089800EB010A294401914FEAFA2585EA8C
:1048D000BA1585EA7A652C4488EA0E050AEA0505C8
:1048E00088EA05052544341D02945BF8240005443C
:1048F000039953F821404FEAF44080EA744080EA7B
:104900009420F41E53F824402044A6F10B0753F8DA
:1049100027104FEAB14484EAF11484EAD104044434
:1049200053F82C002044029943F8210005440199D2
:104930004FEA713C8CEAB10C8CEAB15C00980446F9
:104940000C4001460198084309EA000020436044F6
:104950002A440F9228440B904FEAF22C8CEAB21CA6
:104960008CEA726CC4448EEA0A08039202EA0808D0
:104970008EEA0808C444741D21465BF82440A44410
:10498000069D53F825504FEAF54484EA754484EABD
:104990009524049A53F822502C44A6F10A0853F89F
:1049A00028204FEAB24585EAF21585EAD20525446A
:1049B00053F827402C44049143F8214064444FEAC3
:1049C000703787EAB00787EAB057019901EA000516
:1049D00041EA000C009901EA0C0C45EA0C052F4451
:1049E00009EB040CCDF838C03C440A944FEAFC278C
:1049F00087EABC1787EA7C677744039D8AEA050E3D
:104A00000CEA0E0E8AEA0E0E774406F106095BF8F0
:104A100029502F44029D53F825504FEAF54E8EEA57
:104A2000754E8EEA952E059A53F82250AE44A6F1A3
:104A30000902029253F8225029464FEAB54585EA09
:104A4000F11585EAD105754453F828E0754443F81B
:104A500029502F444FEA743585EAB40585EAB455E8
:104A600000EA040940EA040E019A02EA0E0E49EA3D
:104A70000E09A9440099CD190D954F4409974FEAA5
:104A8000F52E8EEAB51E8EEA756ED644039A82EA3A
:104A90000C0C05EA0C0C82EA0C02724406F10708C1
:104AA0005BF8285002EB050E049953F821504FEAA9
:104AB000F54282EA754282EA952253F826100A44AA
:104AC000A6F1080553F825C04FEABC4585EAFC1558
:104AD00085EADC052A44029D53F825502A4443F810
:104AE000282072444FEA773383EAB70383EAB75347
:104AF00004EA070527433840284318440199114424
:104B00000C91104408900836AFE50023079809E09F
:104B100008AA52F82340991C50F82120224440F85A
:104B200021200133072BF3D9002051B0BDE8F08FCD
:104B30001098000070B506460B4B53F8204000E07B
:104B40000834731C084A52F82330A3420AD9656816
:104B50002368284698470028F2D0002DF0D0002383
:104B6000AB60EDE770BD00BF1099000038B5054699
:104B70000F4C00E010340F4B9C4206D0A368002B72
:104B8000F8D02368AB42F5D110E0094C00E01034B6
:104B9000084B9C4209D0A368002BF8D02168284616
:104BA00001F05CFF0028F2D100E00024204638BD6F
:104BB0005C000020CC00002008B50348034A121A0C
:104BC000002101F090FF08BD08010020142D0020F5
:104BD00008B50648064A121A064901F060FF064A5F
:104BE0000649074801F05BFF08BD00BF0000002038
:104BF000040100207899000000000000789900006E
:104C00000000002008B50B4B01221A700220FFF7AC
:104C100091FF094A09490A4801F092F90320FFF778
:104C200089FFFBF7E7FB074A137B23F001031373AC
:104C300008BD00BF112D0020B89400002899000085
:104C40004C9900000801002008B5FCF77BFE144BCE
:104C500083F30888134C636943F400736361E023B2
:104C600084F822300025E57725766576A576636A97
:104C700043F4E0236362FDF739FEFDF7F9FC4FF0E2
:104C8000FF33A362E3622846FFF754FF0120FFF7DA
:104C900051FF2B462A4629460348FDF7D3FC00BFA7
:104CA000185D002000ED00E0054C000010B5064C3A
:104CB0000020064B9C4206D2204603F034FF002819
:104CC00001DB1C34F5E710BDCC000020CC00002037
:104CD000084681B908B5EFF305833BB9084BDA699B
:104CE0009B689A4202D0FDF739FC03E080F31188FB
:104CF000BFF36F8F08BD81F31188BFF36F8F7047CB
:104D0000DC2C00200A4B834208D04A680B681360F1
:104D10004A685A6000230B604B607047203B9B68D9
:104D20008B42F2D14B7B13F01F0FEED0F5E700BFA3
:104D3000FC2C002038B504460E4D05F1200003F090
:104D400025FFAA68537B13F0200F02D043F008031D
:104D5000537348B15CB9537B13F01F0F07D18369BC
:104D60002BB9044BDA6104E0024BD868F2E7014B3F
:104D7000D86138BDDC2C002038B50546437B13F0E4
:104D80001F0F05D183690BB1002302E0012300E06E
:104D900000230BB3154B53F8204F9C4224D064B131
:104DA0002146284603F0DAFEB8B934B10F4B5B6AEE
:104DB0009C4202D02468002CF1D10C4B03F120025C
:104DC0002A605A6A6A6015605D626B7B63F07F03DC
:104DD0006B730020FFF7AEFF38BD63686B602C601B
:104DE00063681D606560F0E70024D8E7DC2C0020D4
:104DF00038B50446183003F050FF00234FF020026E
:104E0000EFF3118582F31188BFF36F8F10E0637B9E
:104E100043F010036373154B9868A04214BF002041
:104E20000120FFF787FF85F31188BFF36F8F012300
:104E300063B994F90D30002BE9DA21460C48FFF7ED
:104E400061FF637B03F07F036373E0E7074B9B68BD
:104E5000A34200D038BD4FF02003EFF3118083F35D
:104E60001188BFF36F8F03F083FEF3E7DC2C002083
:104E7000FC2C002070B50546036E03B1984705F180
:104E8000180003F00AFF00234FF02002EFF3118611
:104E900082F31188BFF36F8F1FE0012227E02946BC
:104EA0002A48FFF72FFF6B7B03F07F036B7324E02F
:104EB00013F0020F29D0284603F04CFE2946FFF7D5
:104EC00021FF6B7B23F002036B730023AB601CE0BC
:104ED00086F31188BFF36F8F01231A46002B34D15C
:104EE0006B7B13F01F0F02D1A9690029D5D012F0F6
:104EF000010FDDD013F0800FD1D1154B9868A84277
:104F000014BF00200120FFF715FF6B7B43F008035F
:104F10006B7305F130032C6BA342D9D0002CD7D092
:104F200004F1180003F0B9FE204603F013FE2146F9
:104F3000FFF7E8FE637B23F0020363730023A360A3
:104F4000E3672046FFF718FFE3E770BDFC2C002065
:104F5000DC2C002038B5B1F1FF3F08BFB0F1FF3FB6
:104F60001AD003F0F9FD0446C5176901430141EA6F
:104F7000D062181A62EB05039A0042EA907281002F
:104F80001346081945EB0303DA0042EA5072C100E8
:104F9000C80B40EA424038BD034B9868FFF728FF32
:104FA0004FF0FF30F7E700BFDC2C0020014B986882
:104FB000704700BFDC2C002038B504464FF02003BA
:104FC000EFF3118583F31188BFF36F8F03F0FBFDBF
:104FD00040B10022C26703F0E0FD29460648FFF712
:104FE00077FE38BDA368E268934203D001221344E0
:104FF000A360F2E70022FAE7042D0020034B1868B3
:10500000984200D070470020FCE700BF5400002009
:1050100030B1044A5268904201D0006870470020C5
:10502000704700BF5400002008B5044B1B680BB14B
:10503000002008BDFDF7C0F9FBE700BF042D0020EC
:10504000F8B54FF02003EFF3118583F31188BFF318
:105050006F8F284B1860FFF7D1FF044650B3D0E99B
:105060000467244B1B68D917B94208BFB34221D348
:10507000214AD2E90001801941EBE671C2E9000141
:105080009B1B1C4A136000220023C4E90423204612
:1050900003F0DEFD85F31188BFF36F8FA368204610
:1050A00098474FF02003EFF3118583F31188BFF386
:1050B0006F8FD0E744B10F4B1968D4E90423521A1B
:1050C00063EBE173C4E904230B480A490C68D0E997
:1050D0000023121943EBE473C0E9002300240C60A1
:1050E00003F0CEFD2146FDF739F985F31188BFF3B2
:1050F0006F8FF8BD042D00208801002010B5064CEC
:10510000064B9C4206D2A2686168204603F0E3FD8C
:105110001434F5E7002010BDCC000020CC000020A6
:1051200070B582B0044601A90079FBF7F1F9A568D2
:10513000019B1D4423681C892E194FF02002EFF3B8
:10514000118382F31188BFF36F8F01F0C7FBFCF767
:105150006FFA2B5983F30888002383F3148873684C
:10516000984702B070BD19B1012903D102207047E0
:10517000012070476FF015007047FF20704770B531
:1051800016461D4601F02FFA50B90021A94205D25A
:10519000745CFF2C06D10131C9B2F7E7012001E0B0
:1051A0004FF0FF3070BD2DE9F0439DB01546994694
:1051B000249FDDF89480279C01A803F09FFB002129
:1051C00001A8FFF791F814B1289B002B06DC2B896E
:1051D000EE6833446E891E44002513E01A462146CA
:1051E00001A803F091FBF2E723463A4629464846D8
:1051F00001F0F9F9034688B92246394601A803F0BF
:1052000083FB2544B54204D2741B4445ECD9444683
:10521000EAE7269901A803F0BAFB002318461DB05F
:10522000BDE8F0832DE9F04383B000284AD00C4656
:10523000174699460646002947D0002A48D00D89CE
:10524000CB681D4404230DEB03022946384601F0C8
:10525000CAF9804600283ED1BDF8042046F608135E
:105260009A421ED06389002B3BD1BDF8042046F63C
:1052700007139A4238D134607760A6F808909DF8F9
:105280002830B37263892B44F36063892B44BDF8E3
:1052900006201344736104353561404603B0BDE810
:1052A000F0836389BDF806108B4217D104230DEB00
:1052B00003022944384601F096F90028D5D04FF072
:1052C000FF38EAE74FF0FF38E7E74FF0FF38E4E751
:1052D0004FF0FF38E1E74FF0FF38DEE74FF0FF38DF
:1052E000DBE74FF0FF38D8E74FF0FF38D5E700286D
:1052F0004DD0F0B583B00F4616461D4604460368F0
:10530000002B48D043680BBB4FF0FF313AE0042339
:105310000DEB03022169606801F065F90146002880
:105320003CD1A37A1BB12269E3689A4239D223891E
:105330004FF6FF72934217D0BDF80420934213D06A
:10534000BDF80600236918440430206120696369B0
:1053500098421AD223685B89002BD8D0E368834235
:10536000D5D104302061D2E715B1BDF804302B80CF
:10537000236904333B60BDF806303380226913444F
:1053800004332361084603B0F0BD0121FAE74FF072
:10539000FF31084670474FF0FF31F3E74FF0FF3120
:1053A000F0E70121EEE72DE9F04184B004460E4616
:1053B0001546302303AA2946304601F051FFA8BB09
:1053C0003368039A1344AB4233D104F108073A46D9
:1053D0002946304601F057FF28BB04F11408424625
:1053E0002946304601F04FFFE8B9384602F053FA3B
:1053F00060603368AB421FD1CDF804800022009278
:1054000013463946204603F0F4F9C0B92046FEF7AA
:10541000FFFE0546B0B9384602F03DFA6060284606
:1054200004B0BDE8F0816FF00205F8E74FF0FF35FA
:10543000F5E76FF00105F2E76FF00305EFE76FF0B6
:105440000405ECE76FF00505E9E7F0B5A5B0064601
:105450000F4600230893DF2407E025462A466946C5
:10546000304601F01CFB2E44641B002C1DDD09A8F6
:1054700003F044FA002109A8FEF736FF202239463E
:1054800009A803F041FA042208A909A803F03CFA8C
:10549000694609A803F07BFA9DF8233001338DF8A3
:1054A00023301F2CD9DD2025D8E725B0F0BD0128F9
:1054B00000D170470220FCE72DE9F04383B0064697
:1054C000884617461C4601F00BF9082C20D80546E3
:1054D000082802D94FF0FF301CE03046FFF74DFEA0
:1054E0008146A54200D2254622463946684601F04B
:1054F000D6FA2A1B49460DEB040001F0F4FA2B46BC
:105500006A464146304601F08DF818B1012001E0AD
:105510004FF0FF3003B0BDE8F08300B583B08DF8E5
:105520000420012301AAFFF7C7FF03B05DF804FBC5
:1055300004280AD0052803D1481E18BF012070474F
:10554000884214BF0020012070470120704700EB03
:105550004000C001704708B5FFF7F9FF303008BDC3
:105560000B78013BDBB2012B02D84FF4C0707047BF
:105570004FF0FF30704710B5044601F0B1F8FFF767
:10558000EAFFA368181A10BD80682838704730B544
:1055900087B005460C468168102302AA1039FFF730
:1055A000EEFD00284ADB01283CD103232370284666
:1055B000FFF7EAFF014601230DF107022846FFF736
:1055C000DEFD00283DDB9DF8073003F00F0262701E
:1055D0001B092371012801D0042A03D90123637018
:1055E00000232371A9680123A21C20392846FFF754
:1055F000C6FD002827DB012819D0A078FFF757FF48
:10560000A070A9680123E21C18392846FFF7B7FDEE
:1056100000281ADB01280DD0E078FFF748FFE07082
:1056200000200CE002A8FBF72DF92070BFE7032350
:10563000A370E6E70323E370002000E0012007B039
:1056400030BD0120FBE70120F9E70120F7E710B5A5
:1056500082B00C4601A9C0B2FCF76AFC18B1012463
:10566000204602B010BD21460198FFF790FF044686
:10567000019800F0B7FFF3E730B583B00C4601A9FD
:10568000FBF70CF9054610B1284603B030BD019D6B
:105690002846FFF779FF04232246A0F10801284697
:1056A00000F0A1FF0546019800F09CFFECE708B56B
:1056B000816801222039FFF730FF08BD08B58168F5
:1056C00001221839FFF729FF08BD10B582B0044642
:1056D00041EA02118DF80710FFF756FF014601233A
:1056E0000DF107022046FFF7E7FE02B010BD10B52E
:1056F00082B004460191FFF747FF04230DEB03023C
:10570000A0F108012046FFF7D7FE02B010BD08B592
:10571000006A00F0E5FF08BD2DE9F04182B00646C1
:105720000C4617460020FFF71EFD01A9C0B2FCF78A
:10573000FFFB40B14FF00108019800F053FF4046D5
:1057400002B0BDE8F0812C2303FB04631D89DB68F4
:105750001D4404236A462946019800F044FF804610
:1057600040BB2C2101FB04646489BDF8002046F68F
:1057700008139A420CD004BBBDF8002046F607136C
:105780009A421DD12544BDF802301D443D60D3E747
:10579000BDF802108C4202D04FF00308CCE704237E
:1057A0006A462944019800F01EFF0028E4D04FF01B
:1057B0000108C1E74FF00108BEE74FF00308BBE75F
:1057C0004FF00308B8E7F0B583B007460C46002059
:1057D000FFF7C9FC01A9C0B2FCF7AAFBD0B9064685
:1057E0000198FFF7CAFC0546019800F0FBFE2C214A
:1057F00001FB04710023032B05D8CA5C954207D135
:105800000133DBB2F7E701233BB1304603B0F0BD13
:105810000023F9E74FF0FF36F7E74FF0FF36F4E7E4
:1058200010B582B00346084680220192012905D0B6
:1058300002290ED11A6D03F1540402E05A6A03F1F1
:10584000280401A9FCF788FB08B9019B236002B07A
:1058500010BD0120FBE738B504460121FFF7E0FF4A
:1058600010B10125284638BD02212046FFF7D8FF98
:10587000054608B10125F5E72046FFF748FFE0653A
:10588000F0E7F8B505460F4616460024012C10DC5B
:1058900033462C2202FB045221462846FBF71EFC0D
:1058A000034608B90134F1E7002C03DD17B90023E2
:1058B00000E000231846F8BD70B505460E460020EE
:1058C000FBF730F80446022805D0042803D003284B
:1058D00001D0204670BD324601212846FBF7E8F88A
:1058E000012803D00028F4D00524F2E70446F0E7AD
:1058F000002383718360C3600123437103600371DC
:10590000C37170474379012B01D0002070470368B1
:10591000012B01D0002070470379012B01D000201A
:1059200070470120704738B50546FBF725F995F813
:105930005840E31EDBB2012B0DD9022C03D0042CFE
:1059400001D0032C06D1002000F0D8F810B1FF23BD
:1059500085F8583038BD002000F0E3F80028ECD07E
:10596000FF2485F85840EAE770B584B004460E4637
:1059700003A90120FCF7DCFA30B10124039800F000
:1059800031FE204604B070BD0398FFF7F4FD0546D4
:10599000E16D304600F0E5F82C18039800F0A0FE09
:1059A00005460398FFF7E9FB0146082201A801F02C
:1059B0009AF833798DF804302B4601AA21460398D2
:1059C00000F030FE04460028D8D00124D6E708B500
:1059D00000F058FE08BD2DE9F04706460F460021AD
:1059E0000846FFF7C0FB044601210020FFF7BBFB80
:1059F0003B789C4223D0984223D1012399462C2204
:105A000002FB03639C6A013CF06DFFF7A4FD804636
:105A100000252C2303FB09635B6A03EBC402D2F865
:105A200004A053F834101B685246C91A3846FFF7D1
:105A3000CEFF013C5544A845EBD8BDE8F0870023D4
:105A4000DCE70120F9E730B583B00C46154669461E
:105A50000220FFF7FCFDE97901290DD19DF8033003
:105A6000012B0ED0A9682046FFF741FE2046FAF729
:105A70004BFF002003B030BD00222046FFF725FE7B
:105A8000ECE72046FFF71AFEECE770B582B0064659
:105A90000D46FBF779FC0446E86060B3022829D183
:105AA00001A90120FCF744FA08B1012423E02A46A9
:105AB00031460198FBF76EFB044618B1019800F0DF
:105AC00091FD18E00198FFF75FFD014601230DF1FC
:105AD00003020198FFF753FB012806D09DF803301D
:105AE00003F00F03EB710446E8E701238DF8033060
:105AF0002046F3E70724204602B070BD10B582B0FF
:105B000001A90120FCF714FA18B10124204602B0C3
:105B100010BD0198FFF7CBFD0446019800F062FD2F
:105B2000F4E710B584B003A90120FCF701FA18B11D
:105B30000124204604B010BD01A90398FFF727FDFA
:105B4000044660B99DF80730032B03D0039800F09A
:105B500049FDEEE70398FFF7B1FD0446F6E701249F
:105B6000F4E730B44379012B10D0022201FB02F498
:105B7000012B0DD0CD010379013B0268013A02FBF4
:105B800004F201FB0321481930BC70470122EDE704
:105B90000025F0E7024658B1436803F00303012BE8
:105BA00003D0032B07D1036843B1002090607047F6
:105BB0006FF0150070476FF0150070476FF015001B
:105BC00070470346426802F003028160032A03D152
:105BD000006800225A6070470020FAE700207047F2
:105BE00070B584B09DF82040E51E18BF0125012C3A
:105BF0000AD02024099E0396029401951024009453
:105C0000FBF736FD04B070BD3024F3E770B584B007
:105C10009DF82040E51E18BF0125012C0AD0202444
:105C2000099E0396029401950A240094FBF720FD37
:105C300004B070BD3024F3E701207047C80F7047EF
:105C40002DE9F04F87B006460D4614460593002710
:105C50004FF0FF3ABB46B84602E02946B047013450
:105C60002078002800F06981B8F1000F08D12528BC
:105C7000F3D100274FF0FF3ABB464FF00108EEE7A3
:105C80000246A0F12503552B00F24581DFE813F011
:105C90003D014301430143014301430143014301EA
:105CA0004C014301430156005D005D005D005D0055
:105CB0005D005D005D005D005D0043014301430147
:105CC00043014301430143014301430143014301B4
:105CD00043014301430143014301430143014301A4
:105CE0004301430143014301430143014301430194
:105CF000430143014301E2004301430143014301E6
:105D0000430143014301430143014301340187003F
:105D100043014301430170008700430143017000C8
:105D2000430143014301D800430143010F014301F3
:105D3000870043014301E20043017000BAF1000F04
:105D400003DABBF1000F00F0F280BAF1000F0CDBB8
:105D50000AEB8A0A02EB4A0AAAF1300ABBF1000FE9
:105D60007FF47DAF4FF0020B79E7A2F1300AF5E73F
:105D700068280BD06C280ED05FB129462520B0478B
:105D800029462078B0474FF0000868E7682FF1D126
:105D90004820074663E76C2FEED14C20F9E77A2FB5
:105DA0000BD06C2F2ED04C2F34D0059B1A1D059292
:105DB0001B6898464FEAE37906E0059B1A1D059299
:105DC0001B6898464FEAE3792378752B0DD040463F
:105DD0004946FFF733FF40B129462D20B047D8F19F
:105DE000000869EB49090AF1FF3ACDF804A0CDF8A3
:105DF00000B042464B4629463046FFF707FF4FF0BA
:105E000000082CE7059B1A1D05921B6898464FEA6F
:105E1000E379D9E7059B073323F0070303F1080271
:105E200005921A685B680392049329463046FFF78F
:105E300003FF00287ED0DDF80C80DDF81090C3E76A
:105E400029463020B04729467820B0474FF0080A4D
:105E50004FF0010B2378702B09D06C2F17D04C2FEB
:105E60001BD0059B1A1D05921A68002304E0059BB0
:105E70001A1D05921A680023CDF804A0CDF800B0D1
:105E800029463046FFF7ACFE4FF00008E7E6059BD9
:105E90001A1D05921A680023EEE7059B073323F0CD
:105EA000070303F1080205921A685B68E4E7059BA3
:105EB0001A1D0592D3F80090C84603E008F10108C6
:105EC0002946B04798F800000028F7D1BBF1030F2E
:105ED00002D04FF00008C2E6A8EB0903AAEB0303C7
:105EE00003E029462020B047434603F1FF38002B4A
:105EF000F7DC4FF00008B2E6059B1A1D0592294613
:105F00001868B0474FF00008A9E629462520B04799
:105F10004FF00008A3E629462520B04729462078FF
:105F2000B0474FF000089AE64FF0030B97E64FF0AA
:105F3000010B94E64FF0000891E607B0BDE8F08F42
:105F40000FB400B583B004A951F8040B0191FBF71D
:105F50000BFC03B05DF804EB04B0704701F00703DD
:105F6000018B21F007011943018370472DE9F041AE
:105F700006460F469046816819B10C4631B10C684F
:105F800004E00C4602E0234621461C4659B14D6808
:105F900043463A463046A847002CF4D02346002C0E
:105FA000F2D02368F0E7BDE8F081038B13F007031C
:105FB00003D102680AB103207047022B03D0012BE2
:105FC00006D000207047428B002AF8D10420704789
:105FD00003680BB1052070470020704738B50446B0
:105FE0000D46038B002A07DB03F007035A1F012A23
:105FF0000ED9042B32D038BDD0E9000185E803006A
:1060000000232360636001212046FFF7A7FFF2E72A
:10601000D0E9000185E80300002222606260062BBF
:1060200017D12B683BB1628B01326283002BF9D010
:106030001B68002BF6D102212046FFF78FFF204678
:10604000FFF7B3FF0028D6D0238B43F02003238330
:10605000D1E700212046FFF781FFF0E70021FFF79D
:106060007DFF2046FFF7A1FF0028C4D0238B43F01B
:1060700020032383BFE758B110B50C4659B1081D62
:10608000FFF788FD18B9A36833F0030306D110BDEC
:106090006FF0150070476FF01500F8E76FF015000E
:1060A000F5E72DE9F04107460C4616461D46194610
:1060B000201DFFF786FD28B180462B46324621463B
:1060C0003846C047BDE8F0812DE9F84381460C46CB
:1060D00090461F4605E065603B4642464846FFF74E
:1060E000E0FF216829B10D68256066688E42F3D112
:1060F000F1E7BDE8F88310B54FF02004EFF311820B
:1061000084F31188BFF36F8F41610121FBF73CFBE2
:1061100010BD034668B179B10A6882B14A688AB194
:106120000020186058609860D860586198611961C3
:1061300070476FF0150070476FF0150070476FF0F3
:10614000150070476FF015007047F8B504460F460C
:10615000FFF791FF061E37DB4FF02003EFF31182AC
:1061600083F31188BFF36F8F258B05F00705638BD1
:106170004FF6FF718B422FD02E46022D0CD08DB1E1
:10618000042D0FD0062D0DD0052D1FD06FF0040665
:1061900000210B4608460AE00133638301210023F6
:1061A000184604E0B5FA85F35B090021012028B107
:1061B000002038606068A8B107606760ABB982F3FF
:1061C0001188BFF36F8FA9B93046F8BD6FF0220672
:1061D00000210B460846EAE76FF00A0600210B464D
:1061E0000846E4E767602760E8E702212046FBF7FE
:1061F000CBFAE9E700232A4639462046FFF751FF4C
:10620000E2E770B4131D50F82330D3B9012303FA29
:1062100002F4C3682343C360043240F8221000EB49
:10622000C1038268B2F5004F07D399608268B2F566
:10623000004F04D3D96070BC70479980F6E7D980CD
:10624000F9E700EBC3048668B6F5004F18D3A268DF
:1062500000EBC105B6F5004F14D3AA608668B6F509
:10626000004F11D3EB6000EBC2028368B3F5004F1F
:106270000CD3D1608368B3F5004F09D3A160DAE78E
:10628000A288E5E7AA80E9E7EB80ECE7D180F1E7B7
:10629000A180D0E708B58368B3F5004F07D300EBC2
:1062A000C10252685208012A02D0002200E00022F6
:1062B000A2B900EBC102B3F5004F10D352685208E7
:1062C000B3F5004F0DD308230833A2EBD3020132FC
:1062D000B2FA82F2C2F11F02FFF793FF08BD5288A3
:1062E000EDE70423F0E7F8B50346B2F5802F2ED38F
:1062F0000825551BC81D20F007000D4425F0070593
:106300002D1AEF080646186000220023C0E900237A
:1063100087600023C360B7F5004F1AD30823083302
:10632000A7EBD3030133B3FA83F3C3F1200CC3F11A
:1063300024039B0003F1070E4FEADE0100236345AF
:1063400009DA1A1D002446F822400133F7E7042534
:10635000CFE70423E3E74B00B7F5004F2ED34360AC
:10636000B7F5004F2CD3436843F0010343607A1A1A
:1063700056002EF00703C418B7F5004F25D366600A
:106380008468B4F5004F22D3C15025F007030544BB
:106390008468B4F5004F1CD300246C608468B4F5A5
:1063A000004F19D3C2508368B3F5004F16D36B6802
:1063B00043F001036B60FFF76DFFF8BD4380CFE74B
:1063C000438843F001034380D1E76680D8E7C15298
:1063D000DBE700246C80E1E7C252E4E76B8843F01E
:1063E00001036B80E7E770470020704708B5FBF7B3
:1063F000F9FF08BD0EB400B582B003AA52F8041B21
:1064000001920023FBF76CFA02B05DF804EB03B0D5
:10641000704708B5FBF7D2FA002008BD00B583B07D
:1064200001900B684A685268012101A89847002032
:1064300003B05DF804FBF8B507460D4614461E464A
:10644000324621462846B8470544241AF8D1F8BDFB
:106450000022037813B101301A46FAE70A2A14BF62
:1064600000200120704708B513460122FBF75AFBB4
:1064700008BD08B513460022FBF754FB08BD38B52C
:1064800005460C4601F00101FFF7F3FF21462846BF
:10649000FBF75EFB38BD2DE9F04383B0044615469B
:1064A0009DF8286001F00109C1F3C00811F002074E
:1064B00013D1324649462046FFF7D5FF0196BDF875
:1064C000303000939DF82C302A4641462046FBF799
:1064D000B1FB384403B0BDE8F0831A46FBF7DCFAA1
:1064E0000746E6E710B504464268536812688168BB
:1064F0000068FFF7A0FF636800221A6010BDF8B5BE
:1065000007460E4615460024B44206D2395DAB68F4
:106510005B68284698470134F6E73046F8BD0068C6
:106520004B6898420BD310B48C682344984209D22C
:1065300008694B69984209D2002010BC70470120BD
:1065400010707047002313700120F6E76FF00B0303
:106550008B61002313700120EFE770B582B0054610
:106560000C46CE680DF10702FFF7D9FF80B92B6802
:10657000616822695B1A46F83230236906EBC3066C
:106580006B687360236901332361012002B070BD21
:106590009DF80700FAE7F8B50D4617461E46069C1B
:1065A0002060FBF7ADFCB8B1436863608368A3600B
:1065B000E760002222612B686361A261C068FEF778
:1065C000D5FA60B12246314600F0DDFBA3690BB974
:1065D00023692B60A069F8BD6FF01500FBE76FF031
:1065E0001200F8E77047F8B504460D4617461E46F8
:1065F00083688B4204D3721893420ED2002300E0CA
:10660000002363B1E068FEF7B1FA6168294483684A
:106610001C6833463A46A047F8BD0123F1E76FF006
:106620001500F9E72DE9F84305460E4691461F4649
:1066300083688B4204D37A1893421ED2002300E071
:106640000023E3B1E868FEF791FA04468368DB684B
:1066500000219847804668B969683144A3685D683D
:106660003B464A462046A8478046A368DB6801218E
:10667000204698474046BDE8F8830123E1E76FF0E4
:106680001508F7E72DE9F04105460E4617468368E1
:106690008B4204D30A4493421DD2002300E000231E
:1066A000DBB1E868FEF762FA04468368DB68002124
:1066B0009847804660B969683144A3689B683A4648
:1066C000204698478046A368DB680121204698470A
:1066D0004046BDE8F0810123E2E76FF01508F7E7D7
:1066E00008B5C068FEF742FA83681B6998470078CE
:1066F00008BD00F180431A683AB14FF08042D2F8E9
:10670000042311420CD0012200E0002210464AB1BD
:1067100082B000221A601B680193019B02B070478F
:106720000022F3E770474FF080430322C3F80423AD
:106730007047C06801EB4101890038310844704757
:10674000406801EB410100EB81007047C068C1EB7C
:10675000C10100EB8100704708B5C9B2FFF7E9FF3E
:10676000806800F0070008BD4FF02003EFF31182AE
:1067700083F31188BFF36F8F036813F0C00301D058
:106780008B4207D101230360002082F31188BFF3FD
:106790006F8F70474FF0FF30F7E710B44FF02003D2
:1067A000EFF3118283F31188BFF36F8F036803F057
:1067B000C00403F00703012B09D08C420AD04FF02C
:1067C000FF3082F31188BFF36F8F10BC70470160F8
:1067D0000020F6E76FF00F00F3E74FF02003EFF330
:1067E000118283F31188BFF36F8F036803F0C00336
:1067F00043F00203036082F31188BFF36F8F704789
:10680000F8B506460C46FFF794FF05684768002375
:1068100040F8083BFFF7E1FF1DB13A4621463046FC
:10682000A847F8BD4FF0804301221A60704770B549
:1068300006461546CCB22146FFF77BFF29460830B5
:10684000FFF792FF002806DB21463046FFF778FF6E
:1068500043689847002070BD08B58022FFF7E7FF26
:1068600008BD2DE9F041074616461D465FFA81F83E
:106870004146FFF75EFF044629460830FFF78DFFCB
:1068800000280ADB73682360B368636041463846BA
:10689000FFF756FF036898470020BDE8F08108B570
:1068A0008023FFF7DEFF08BD6FF02200704710B5B0
:1068B0001446C9B2FFF74AFF0021A04710BD4FF0B0
:1068C0008042D2F8183403F00303D2F8182412F4EB
:1068D000803FF4D09842F2D1704770477047401A19
:1068E00020F07F40704710B504460230FBF7A4FC4F
:1068F000FBF7D4FCA04206D0FBF7D0FC04460230E4
:10690000FBF79AFCF4E710BD38B50446FBF7C6FC6C
:10691000054601462046FFF7E2FF01280DD020463C
:10692000FBF78AFCFBF7BAFC05460146A01EFFF701
:10693000D6FFB0F5000F04D238BD2846FFF7D3FFCD
:10694000FAE72846FFF7CFFFF6E710B50446FBF756
:1069500095FCFBF7BBFC2046FFF7D6FFFBF796FC48
:1069600010BD08B5FBF756FD08BD08B5FFF7F9FFE8
:10697000002008BD08B50021012000F005F808BD81
:1069800008B5FBF7FDFF08BD08B502F0B2F808BD79
:1069900008B501460068FFF7F7FF08BD08B5FBF72B
:1069A0006DFEFBF7ABFF08BD0020704708B5002364
:1069B0001370CB1E032B12D8DFE803F002060A0E79
:1069C0001146FBF717FF08BD0021FBF7B3FEFAE7FE
:1069D0000021FBF7D3FEF6E7FBF7FAFEF3E7002012
:1069E000F1E743685A1E134206D11F2B06D90368EC
:1069F0001A4205D0002070470020704700207047E1
:106A00000120704700B585B00B6801934B688A6818
:106A1000202B12D9B3F1004F11D8013BB3FA83F305
:106A2000C3F11F035B0003F03E031343039301A96B
:106A3000FBF7D4FF05B05DF804FB0823F5E73E2320
:106A4000F3E708B5FCF72AF808BD02460B781BB13E
:106A500002F8013B0131F9E71370704703780A78B7
:106A6000934203D113B101300131F7E7981A70470F
:106A70007AB1531E0FD010B404780A78944203D12F
:106A800001300131013BF7D100780B78C01A10BCFE
:106A900070470020704700780B78C01A704710B418
:106AA00080EA010313F0030F01D0034617E0034609
:106AB00013F0030F0BD0A2B111F8014B03F8014BF7
:106AC000013AF5E751F8044B43F8044B043A032A22
:106AD000F8D804E011F8014B03F8014B013A002A01
:106AE000F8D110BC704710B4CCB2034613F0030FBA
:106AF00004D09AB103F8014B013AF7E7C9B241EA71
:106B0000012141EA0141032A06D943F8041B043A52
:106B1000F9E703F8014B013A002AFAD110BC70479B
:106B20004FF0FF30704708B5FDF700F808BD436827
:106B30005B68D3F810350B600020704743685B68D2
:106B4000D3F8040542400A404240C3F8042500201F
:106B5000704743685B68C3F80815002070474368B6
:106B60005B68C3F80C150020704743685A68D2F878
:106B700004354B40C2F804350020704770B4C0683B
:106B8000051D4368DBB10E4600240AE00B68436034
:106B90006C68A1420FD16B600DE06C600BE01C468D
:106BA0001B685BB19E42FAD1002CEFD00B682360CA
:106BB0006B689942F1D000230B6000E052B162B1E2
:106BC00043680B6041606B680BB1002006E06960B0
:106BD000002003E06FF0150000E0002070BC70475B
:106BE000002070474B6803444B600B6803440B6004
:106BF0008B68181A8860704738B5044600F0C0FAF0
:106C000005466068FDF796F8A3685B1BA3606268A1
:106C10002A446260002BF4D1002038BD00B585B055
:106C2000002301930290039101A8FFF7E5FF05B04F
:106C30005DF804FB70B50C46154600F0A1FA064657
:106C400000F09AFAA04219D9002C1ADB85421BD811
:106C50002B1998421BD3B4FBF6F306FB1343CBB9B5
:106C6000B5FBF6F306FB1353BBB9AE4201D90020C6
:106C700006E029462046FFF7D1FF01E06FF015003E
:106C800070BD6FF01500FBE76FF01500F8E76FF0CF
:106C90001500F5E76FF01500F2E76FF01500EFE76C
:106CA00010B50446A368032B09D9236819686068E6
:106CB00000F056FA21460420FFF794FFF2E7FCF7B4
:106CC00031FA002010BD00B585B001910290039209
:106CD00001A8FFF7E5FF05B05DF804FB70B50C46B1
:106CE00016461D4600F048FA844215D2002C16DBE9
:106CF000854217D82B19984217D314F0030F17D1D8
:106D000015F0030F17D10DB9002007E02A463146D0
:106D10002046FFF7D8FF01E06FF0150070BD6FF05F
:106D20001500FBE76FF01500F8E76FF01500F5E7C9
:106D30006FF01500F2E76FF01500EFE770B50C4645
:106D400016461D4600F018FAA04210D9002C11DB9F
:106D5000854212D82B19984212D30DB9002008E0B1
:106D60002A4621463046FFF79AFE002001E06FF0E8
:106D7000150070BD6FF01500FBE76FF01500F8E728
:106D80006FF01500F5E72DE9F04786B0894690468B
:106D900083685B6901AA05A9984700242646A24694
:106DA000019B534516D9059F07EBCA077B680393E0
:106DB00000253B68AB420AD902940496414602A8DA
:106DC000C84738B1039B1C4401360135F1E70AF18D
:106DD000010AE5E706B0BDE8F0870B46C26892E815
:106DE000030083E803000020704701207047C26859
:106DF00043681B689168897B11B1D3F8201199B958
:106E000000B583B0D3F8241131B10021C3F82411A7
:106E1000D3F824310193019B926813680BB1516838
:106E2000984703B05DF804FB4FF48071C3F8081372
:106E30000121D960936800229A73704770B582B0BF
:106E400005460C464B79012B06D0032B11D06FF071
:106E50002203184602B070BD00238DF80630A379D6
:106E6000032B3AD1E37943B1012B10D06FF0220309
:106E7000EFE710238DF80630F1E700238DF804309A
:106E800023795BB1022B24D06FF02203E1E76B681A
:106E90001B792BB301238DF80430F1E700238DF823
:106EA000053021682846FCF72DFC0346D8B96A68EE
:106EB00010689DF805109DF806609DF80420314388
:106EC0000A43C0F86C25EA6894E8030082E80300EE
:106ED000BFE70E238DF80530E3E76FF02203B8E734
:106EE0006FF02203B5E76FF02203B2E70B46C268EA
:106EF00092E8030083E803000020704743681B68A2
:106F0000D3F88004C3F88004704710B483B0C46819
:106F100043681B68D3F810216AB1227C0A700020F4
:106F2000C3F81001D3F810210192019A01221A60CE
:106F300003B010BC70474FF0FF30F9E770B483B076
:106F400043681E68C568D6F82031F3B1AB689889EC
:106F5000904200DB10460023C6F82031D6F82021ED
:106F60000192019A984205DDAA689268CC5CD454DB
:106F70000133F7E7AB689B68C6F84435C6F84805A7
:106F80000123B36003B070BC70470020FAE7436888
:106F90001B68C068D3F810216AB182B00022C3F820
:106FA0001021D3F810210192019A027C0A7001206D
:106FB000186002B070470020704743681B68C268C1
:106FC0009268002191734FF48072C3F804237047D4
:106FD000C3689B6801229A73704743681A68C36844
:106FE0009B689B7B4BB9D2F8203143B1D2F8043374
:106FF00013F4807F05D001207047002070470020E7
:1070000070470020704743681B68D3F810010038B0
:1070100018BF0120704743681B681022C3F804237F
:10702000704743681B681022C3F808237047436801
:107030001B684FF40072C3F80423704743681B6851
:107040004FF40072C3F80823704738B5044643680C
:107050001D68D5F8043313F4807F06D1D5F80433C6
:1070600013F0100F07D1002038BDFFF7B6FF00283E
:10707000F4D00120F8E72046FFF7C5FF0028F3D041
:107080000120F1E701207047C368986801609B68A0
:107090005A607047F0B585B08DF8071043681D68D9
:1070A000C66801F0CBFDC8B906F10C0464270123C2
:1070B000BFF35B8F54E8002F002A03D144E800316E
:1070C0000029F7D1BFF35B8F0AD021200021FDF703
:1070D00041FF013F17F0FF07E9D101E00123F36011
:1070E0000023C5F82031D5F820310393039B0DF11F
:1070F0000703C5F844350123C5F84835AB604FF4A4
:107100007A74D5F8203123B9012000F008F8013C49
:10711000F7D10123EB600023F36005B0F0BD08B5A3
:1071200001F092FD08BD4FF08053186970474FF091
:1071300080535869704710B5FFF7F5FF0446FFF715
:10714000F6FF00FB04F010BD10B50446FFF7EBFF9F
:10715000B4FBF0F300FB1340B0FA80F0400910BD1F
:1071600038B504460D46FCF7C9FD29462046FCF714
:10717000D5FDFCF7BBFD38BD08B5FFF7DCFF08BD4A
:1071800008B5FFF7D0FF08BD08B5FFF7D0FF08BD71
:107190000020704770B40368CD1A002D4BDD1C78B9
:1071A00093F90060002E0BDB5C1C04601B781360FD
:1071B00013680268891A8B424FD8002070BC704750
:1071C00004F07F04013C032C38D8DFE804F0020A05
:1071D0001523012D35DD5B781360036802330360EE
:1071E000E6E7022D30DD5C789B7843EA04231360E8
:1071F000036803330360DBE7032D28DD5D789C78AB
:10720000240244EA0544DB78234313600368043313
:107210000360CDE7042D1DDD5D789C78240444EAED
:107220000564DD7844EA05241B7923431360036871
:1072300005330360BCE76FF05F00BFE76FF06300EA
:10724000BCE76FF05F00B9E76FF05F00B6E76FF083
:107250005F00B3E76FF05F00B0E76FF05F00ADE78E
:1072600038B504680D1B002D07DD25789D4207D138
:1072700001340460FFF78EFF38BD6FF05F00FBE75D
:107280006FF06100F8E730B583B00446154602237D
:1072900001AAFFF7E5FF08B103B030BD019A2168EC
:1072A000284600F0FEFA2368019A13442360F3E7AE
:1072B00002464FF0004300201F2804D8134202D199
:1072C0005B080130F8E7704782B00190002001AA06
:1072D000034605E012F8011B41EA00200133DBB24E
:1072E000032BF7D902B0704708B5FFF7EDFF08BDD3
:1072F000A9B170B5054601F18044013C00EB84045E
:10730000A5420BD82868FFF7EFFF06462068FFF775
:10731000EBFF45F8040B44F80469F1E770BD7047D2
:10732000F0B400231D4685421CD21768FC1A146075
:1073300051F8046BB4422CBF4FF0000C4FF0010C1D
:107340009F422CBF63460CF10103A41B42F8044B7F
:107350000135E8E71168C81A42F8040B99422CBFBE
:1073600000230123002BF5D1F0BC70472DE9F00379
:1073700000240F2840F273810D68A5FB038914EBEC
:1073800008042CBF0125002505EB090716683619EE
:107390002CBF012500253D4416604E68A3FB0667FF
:1073A000AD192CBF012400242744566875192CBF41
:1073B000012400243C4455608E68A3FB0678E41940
:1073C0002CBF01260026464495682D192CBF0124A8
:1073D000002434449560CE68A3FB0678E4192CBFE2
:1073E000012600264644D5682D192CBF012400240F
:1073F0003444D5600E69A3FB0678E4192CBF01263E
:107400000026464415692D192CBF0124002434445C
:1074100015614E69A3FB0678E4192CBF01260026EE
:10742000464455692D192CBF01240024344455616C
:107430008E69A3FB0678E4192CBF0126002646447A
:1074400095692D192CBF0124002434449561CE691F
:10745000A3FB0678E4192CBF012600264644D56913
:107460002D192CBF012400243444D5610E6AA3FBDE
:107470000678E4192CBF012600264644156A2D190A
:107480002CBF01240024344415624E6AA3FB067805
:10749000E4192CBF012600264644556A2D192CBF3D
:1074A00001240024344455628E6AA3FB0678E41953
:1074B0002CBF012600264644956A2D192CBF0124B5
:1074C000002434449562CE6AA3FB0678E4192CBFED
:1074D000012600264644D56A2D192CBF012400241C
:1074E0003444D5620E6BA3FB0678E4192CBF012649
:1074F00000264644156B2D192CBF0124002434446A
:1075000015634E6BA3FB0678E4192CBF01260026F9
:107510004644556B2D192CBF012400243444556377
:107520008E6BA3FB0678E4192CBF01260026464487
:10753000956B2D192CBF0124002434449563CE6B28
:10754000A3FB0678E4192CBF012600264644D56B20
:107550002D192CBF012400243444D5631038403247
:10756000403106E70D68A5FB038914EB08042CBF26
:107570000125002505EB0907166836192CBF0125E2
:1075800000253D4416604E68A3FB0667AD192CBF6D
:10759000012400242744566875192CBF01240024B7
:1075A0003C4455608E68A3FB0678E4192CBF012685
:1075B0000026464495682D192CBF0124002434442C
:1075C0009560CE68A3FB0678E4192CBF012600263F
:1075D0004644D5682D192CBF012400243444D560BD
:1075E0000E69A3FB0678E4192CBF01260026464449
:1075F00015692D192CBF01240024344415614E69EE
:10760000A3FB0678E4192CBF0126002646445569E1
:107610002D192CBF01240024344455618E69A3FB2D
:107620000678E4192CBF01260026464495692D19D9
:107630002CBF0124002434449561CE69A3FB067855
:10764000E4192CBF012600264644D5692D192CBF0C
:10765000012400243444D561083820322031072821
:1076600080D890B151F8046BA6FB0378E4192CBFC5
:1076700001260026464415682D192CBF012400243C
:10768000344442F8045B0138EBE71368234442F8C2
:10769000043B2146A3422CBF002401248B42F4D397
:1076A000BDE8F00370472DE9F0411E46BAB104462B
:1076B00088461746824212D9002308462146F8F729
:1076C0001FFD0446012908BF002801D34FF0FF34F5
:1076D00016B107FB148737602046BDE8F08116B16C
:1076E0004FF0FF3333604FF0FF30F6E710B48B6894
:1076F0001C68A31C5B0003F008032344202106E060
:1077000004FB03F2C2F1020202FB03F3490807295A
:10771000F6D85B42036010BC704708B58900FCF7DF
:1077200003FD08BD012303600023436083607047AD
:1077300078B110B50446806828B16168FFF7EDFFA5
:10774000A068FCF7DFFC0123236000236360A360D3
:1077500010BD704742F2107399421ED870B50446AE
:107760000D4643688B4201D3002070BD042128469A
:10777000FCF7C0FC064698B1A16851B1626892005E
:10778000FFF78DF96168A068FFF7C7FFA068FCF7F5
:10779000B9FC6560A6600020E7E76FF00F00704756
:1077A0006FF00F00E1E7F8B588422CD006460D4691
:1077B0004B683BB1013B4BB1AA6852F823202AB970
:1077C000013BF8E7FFF7B4FF00271AE05C1C2B68C9
:1077D00033607268A24206D221463046FFF7BAFFF4
:1077E000074648B10DE0B068121B9200002100EB83
:1077F0008400FFF778F90027A200A968B068FFF7B6
:107800004EF93846F8BD0027FBE770B504460D4633
:107810000121FFF79FFF064608B1304670BD626840
:1078200092000021A068FFF75EF9A36885EAE5727F
:10783000A2EBE5721A60002D02DB01232360ECE766
:107840004FF0FF33FAE74368B1EB431F0AD2836876
:107850004A0953F8220001F01F0120FA01F101F05A
:1078600001007047002070470246406890B110B593
:10787000441E2CB1936853F824300BB9013CF8E74F
:10788000936853F82400FFF713FDC0F1200000EBCC
:10789000441010BD704708B5FFF7E6FF0730C00879
:1078A00008BD2DE9F84305460F46164612F00303BE
:1078B00018BF012303EB9204C2EB84094368A3427F
:1078C0000AD0FFF735FF2846FFF72CFF2146284650
:1078D000FFF740FF804680B900212846FFF795FF5B
:1078E000804650B94FB1A868324639464844FFF740
:1078F000D6F82146A868FFF7FBFC4046BDE8F883B0
:10790000F8B50646084673689F00B2EB830F0FD8A0
:107910001346BB4213D2B46823F00301645803F04A
:107920000305ED00EC4014F0FF0F1AD10133F0E72E
:10793000D21B8C180021FFF7D6F820463A460023C8
:107940000BE0B46823F00301655803F00301C9009C
:10795000CD40D41A013C055501339A42F1D800209C
:10796000F8BD6FF00700FBE7F8B505460F464C0978
:1079700001F01F06FFF778FF38446B68B0EB431F38
:1079800010D81F2F24D96B68A3421FD9A9681A1BCE
:107990006FF040401F18024451F8222041F8272080
:1079A000013BF1E710F01F0118BF012101EB50115D
:1079B0002846FFF7CFFE0028E3D00BE0A96803F1CB
:1079C0008042013A002041F82200013B002BF5D112
:1079D000C6B90020F8BDA86850F82410C6F12003ED
:1079E00001FA06F240F82420A86850F824203A430F
:1079F00040F82420013421FA03F76968A142EAD84B
:107A00000020E7E70027F8E7F8B54368B3EB511F1C
:107A100025D34C0901F01F07A3421ED01F2936D8D9
:107A2000002F38D042684FF0000C92B3866802F104
:107A30008043013B56F82350C7F1200125FA07F493
:107A400046F82340866856F8234044EA0C0446F87A
:107A50002340013A05FA01FCE7E7002FDED00021C0
:107A6000FFF7D3FE16E08268191952F8211042F888
:107A7000231001334268121B9A42F4D842689A429A
:107A8000CED98268002142F823100133F6E70023A3
:107A9000F0E70020F8BD0020FCE730B4436843B1B4
:107AA000846803F18042013A54F822200AB9013B6C
:107AB000F5E74A6842B18D6802F18044013C55F80F
:107AC00024400CB9013AF5E703B9C2B1934218D882
:107AD00003D24FF0FF3015E0013B73B1846803F12E
:107AE0008042013A54F822408D6855F82220944291
:107AF0000AD8F1D24FF0FF3004E0002002E000206D
:107B000000E0012030BC70470120FBE72DE9F04F79
:107B100083B0914600930C9B5A68D9F80430013326
:107B20009A425AD382468B460C9B9868002857D0BD
:107B300092000021FEF7D7FF0C9B9C68D9F80480C7
:107B4000DBF80430434528BF43460193002620E07C
:107B5000DAF8083053F826702368DBF808100D684F
:107B600007FB0535009B03FB05F53B4622460198C4
:107B7000FFF7FCFB2B462246D9F808104046FFF7DA
:107B8000F5FB44F8047B08F10103002244F82320AC
:107B900001364645DCD308F1010292002146DAF8AD
:107BA0000800FEF77CFF49465046FFF776FF0028A5
:107BB0000ADBDAF80820D9F808104046FFF7B0FBD6
:107BC000002003B0BDE8F08F0C9B9A68DAF808102B
:107BD0004046FFF7A5FB0020F3E76FF00300F0E756
:107BE0006FF00300EDE710B586B001240594029410
:107BF000039405AC0494009313460A4602A9FFF7C8
:107C000085FF06B010BD70B40646436843B1B46842
:107C100003F18042013A54F822200AB9013BF5E70A
:107C20004A6842B18D6802F18044013C55F8244015
:107C30000CB9013AF5E703B94AB393420FD893421E
:107C400010D33068002802DD0A68002A21DB0A68A8
:107C5000002A0BDD002809DA4FF0FF3000E0306821
:107C600070BC704708684042FAE7013B6BB1B468EA
:107C700003F18042013A54F822408D6855F82220E1
:107C80009442EDD8F1D24042EAE70020E8E7002034
:107C9000E6E70120E4E700B585B081EAE173A3EBF4
:107CA000E173009300290BDB01230193012302936D
:107CB000CDF80CD001A9FFF7A6FF05B05DF804FBD5
:107CC0004FF0FF33F1E7F8B507461446904214D061
:107CD000B94205D03846FFF766FD8446002843D1F7
:107CE00001233B6066685EB1A16806F18043013BF9
:107CF00051F8233023B9013EF5E70C460146E7E78A
:107D000031463846FFF726FD844668BBA068BB684D
:107D1000002425460EE050F8041B1A68A4182CBF56
:107D2000012200220C4443F8044B8C422CBF144621
:107D3000541C0135B542EED308E01A68224443F8DA
:107D4000042BA2422CBF00240124013564B17A68BF
:107D5000AA42F2D8691C3846FFF7FCFC844618B9E1
:107D6000BB6803EB8503E8E76046F8BDF0B585B076
:107D700005460E46144611463046FFF78EFE002893
:107D80002CDB01A8FFF7CEFCAC4214D0AE4205D0EC
:107D900031462846FFF707FD0746C8B901232B6087
:107DA000606880B1A26800F18043013B52F8233043
:107DB0004BB90138F5E7214601A8FFF7F4FC074667
:107DC00030B901ACE2E7AA68A168FFF7A9FA002779
:107DD00001A8FFF7ADFC384605B0F0BD6FF009070C
:107DE000F9E7F8B506460C4615460F68136807FB19
:107DF00003F3002B16DA11462046FFF74EFE00284B
:107E000007DB2A4621463046FFF7B0FF70B93760DE
:107E10000CE0224629463046FFF7A8FF30B97F42E2
:107E2000376003E0FFF74FFF00B93760F8BDF8B5E2
:107E300006460C4615460F68136807FB03F3002B34
:107E400017DD11462046FFF728FE002807DB2A46EB
:107E500021463046FFF78AFF00B93760F8BD224659
:107E600029463046FFF782FF0028F7D17F4237606E
:107E7000F4E7FFF728FF0028F0D13760EEE72DE99F
:107E8000F04387B080460E46174603A8FFF74AFC2A
:107E90006846FFF747FCB0450CD0B84512D075686E
:107EA000C5B1B26805F18043013B52F823308BB96C
:107EB000013DF5E7314603A8FFF775FC8146D0B9CF
:107EC00003AEEAE739466846FFF76DFC814690B994
:107ED0006F46E4E77C6844B1BA6804F18043013B33
:107EE00052F823300BB9013CF5E729194046FFF75A
:107EF00031FC814648B16846FFF71AFC03A8FFF73A
:107F000017FC484607B0BDE8F08300214046FFF764
:107F10007CFC81460028EED17CB1D8F8081004F131
:107F20008042013ABB6853F8223001EB8202B1680B
:107F30002846FFF71BFA013CEEE732683B6803FB7B
:107F400002F3C8F80030D6E700B585B001230193ED
:107F50000293CDF80CD0009201AAFFF790FF05B074
:107F60005DF804FB2DE9F04F97B006460F46154625
:107F70001C4600211846FFF78EFE002800F0B7814E
:107F800013A8FFF7CFFB10A8FFF7CCFB0DA8FFF756
:107F9000C9FB0AA8FFF7C6FB07A8FFF7C3FB2146EA
:107FA0002846FFF77AFD002810DA2EB1002130466E
:107FB000FFF72BFC804678B92FB129463846FFF7EA
:107FC000F2FB804640B94FF0000814E0294613A8A0
:107FD000FFF7E9FB804690B113A8FFF7A9FB10A8B3
:107FE000FFF7A6FB0DA8FFF7A3FB0AA8FFF7A0FB6E
:107FF00007A8FFF79DFB404617B0BDE8F08F21466C
:1080000010A8FFF7D0FB80460028E5D1012310938C
:108010001393696802310DA8FFF79CFB8046002886
:10802000DAD100210DA8FFF7F0FB80460028D3D15C
:1080300002210AA8FFF78EFB80460028CCD103213D
:1080400007A8FFF787FB80460028C5D110A8FFF7D7
:108050000BFC00F01F031E2B11D8C3F11F0300936C
:108060009946194613A8FFF77FFC80460028B3D134
:10807000494610A8FFF778FC804610B1ACE7002312
:108080000093149B03F1FF3B119A0192511E029140
:10809000A3EB02094FEA491A514610A8FFF764FC06
:1080A0008046002898D110A913A8FFF7ACFD00283E
:1080B0000EDB0F9A52F82930013342F8293010AA0A
:1080C00013A90846FFF7B3FE80460028EBD083E7EC
:1080D000514610A8FFF798FC804600287FF47CAF3B
:1080E00003960497029F02955D460594019CBD424C
:1080F00040F2CC8015994FEA850951F825004FEAE6
:10810000870A129B53F82720904217D3EB1B03F1E9
:108110008043013B0F9A4FF0FF3142F823100F9A32
:10812000EB1B019303F1804B0BF1FF3B4FEA8B06F6
:1081300052F82B30013342F82B3047E06FF04043C8
:1081400005EB030CDDF83C80EE1B1E44002351F8C8
:108150002C10FFF7A8FA48F82600E0E73A460C9BF7
:108160001A60129B53F80A200C9B5A600F9B9A5975
:108170000AA90846FFF7E8FE804600287FF42CAFE6
:10818000002107A8FFF741FB804600287FF424AFB9
:10819000012D30D905F18043023B159A52F8232076
:1081A000099B1A604DB305F18043013B159A52F8C3
:1081B0002320099B5A60159B53F80920099B9A605C
:1081C00007A90AA8FFF71FFD002818DD0F9A935989
:1081D000013B935100210AA8FFF717FB80460028B6
:1081E0007FF4FAAE002FB9D004F18043023B129A1B
:1081F00052F82320B3E70022D2E72A46D9E70F9BA3
:1082000053F82B2010A90AA8FFF79EFE80460028ED
:108210007FF4E2AE019B5E1E760131460AA8FFF7AD
:10822000A3FB804600287FF4D7AE0AAA13A908460C
:10823000FFF7FDFD804600287FF4CEAE002113A895
:10824000FFF729FD002801DB013D50E710A90AA82E
:10825000FFF7A9FA804600287FF4BEAE31460AA88F
:10826000FFF782FB804600287FF4B6AE0AAA13A966
:108270000846FFF7B6FD804600287FF4ADAE0F9AA2
:1082800052F82B30013B42F82B30DDE7039E049F70
:10829000029D059C66B10DA93046FFF784FA804621
:1082A00000287FF499AE2A68236803FB02F3336049
:1082B000002F3FF491AE009913A8FFF7A5FB80466D
:1082C00000287FF489AE2B68139313A93846FFF773
:1082D0006AFA804600287FF47FAE00213846FFF717
:1082E000DAFC00287FF478AE01233B6074E66FF07F
:1082F0000B0880E670B504460E4615460021104670
:10830000FFF7C9FC002826DB2B4632462146002019
:10831000FFF728FE064668B900212046FFF7BBFCA0
:10832000002809DA2A4621462046FFF75AFD06466C
:108330000028F1D0304670BD29462046FFF763FC87
:108340000028F7DB2A4621462046FFF770FD064647
:108350000028F1D0EEE76FF00906EBE72DE9F04FCA
:10836000ADF2446D07468B4616461D46DDF868960D
:1083700000211846FFF78FFC002840F32D82AB68E0
:108380001B6813F0010F00F02A8200213046FFF72E
:1083900082FC0028C0F2268229460DF23C60FFF7DD
:1083A000A5F90DF5C660FFF7BDF90DF22460FFF7E2
:1083B000B9F906A8FFF7B6F94FF4C062002109A881
:1083C000FEF791FB3046FFF74FFAB0F5287F07D252
:1083D000EF2820D84F2820D8172820D9032400E0E0
:1083E00006246B6803F1010A51463846FFF7B2F9DB
:1083F0008046B0B1631E01259D400123A340AB42DE
:1084000040F2D08105EB450009AB03EB8000FFF79C
:108410008FF90135F1E70524E3E70424E1E70124BE
:10842000DFE751460CA8FFF795F980460028E1D117
:108430004FEA4A010DF22460FFF78CF980460028CC
:10844000D8D1DBF800A0BAF1FF3F46D0B9F1000F58
:108450004FD0D9F80830002B4BD00C2249460DF5EF
:10846000C660FEF71CFB29465846FFF7CCFB0028E8
:1084700066DB2A4659460CA8FFF73CFF80460028D9
:10848000B8D10DF224630093DDF83C362A460DF591
:10849000C6610CA8FFF73AFB80460028AAD10DF56B
:1084A000C6613846FFF77FF980460028A2D10DF259
:1084B0002463DDF83C2629463846FFF794FB8046C6
:1084C000002897D1012C43D87368049300230593A7
:1084D0009B460393A0461C46ADE0594606A8FFF70D
:1084E00062F98046002885D1012306930DF1180B0F
:1084F000ACE701210DF5C660FFF787F9804600283B
:108500007FF478AF696889010DF5C660FFF72CFA32
:10851000804600287FF46EAF2A460DF5C6610846F6
:10852000FFF7E8FE804600287FF464AFB9F1000F42
:1085300099D00C220DF5C6614846FEF7B0FA92E7D5
:1085400059460CA8FFF72FF98046002899D051E72B
:10855000631E03934FF0010B0BFA03F3049303EB39
:10856000430B09AB03EB8B0B696801315846FFF7EE
:10857000F1F8804600287FF43DAF0CA95846FFF77C
:1085800012F9804600287FF435AF0023B046264616
:108590001C46039BA3420ED90DF224630093DDF821
:1085A0003C362A4659465846FFF7B0FA002840F0B4
:1085B000E4800134EDE7049B03F1010B0123B34098
:1085C0005B4529D90BEB4B0409AB03EB84046968C9
:1085D00001312046FFF7BEF8002840F0D1800BF1B2
:1085E000FF3101EB410109AB03EB81012046FFF7AD
:1085F000DAF8002840F0C7800DF224630093DDF81C
:108600003C362A460CA92046FFF780FA002840F0A5
:10861000BD800BF1010BD1E73446464654E70BF120
:10862000010BA8EB0B029340039A1A430392D8451F
:1086300028D0022305932CB9049B002B72D0013B58
:1086400004932024013CB368049A53F82230E34099
:1086500013F0010302D1059A002AECD0002BDED1E1
:10866000059A012ADBD10DF224630093DDF83C3634
:108670002A4639463846FFF749FA0028DBD04446F7
:108680008046B7E64FF0000BC3450ED20DF22463CF
:108690000093DDF83C362A4639463846FFF736FA6D
:1086A000002876D10BF1010BEEE7039B03EB4301AE
:1086B0000DF224630093DDF83C362A4609A800EB4E
:1086C00081013846FFF722FA002865D1012305937E
:1086D0004FF0000BCDF80CB0ADE701345C4526D26D
:1086E0000DF224630093DDF83C362A4639463846BD
:1086F000FFF70CFA002852D1039B5A000392012382
:10870000B3401342E9D00DF224630093DDF83C3608
:108710002A460CA93846FFF7F9F90028DDD034467F
:10872000804667E6049C334646469846D6E734467C
:1087300046460DF22463DDF83C2629463846FFF70D
:1087400052FA804600287FF455AEBAF1FF3F7FF41D
:1087500051AE7368002B3FF44DAEB3681B6813F045
:10876000010F3FF447AE4FF0FF333B603A462946D6
:108770003846FFF736FB80463CE63446804639E60D
:108780003446804636E63446804633E634468046F4
:1087900030E6444680462DE6444680462AE6344686
:1087A000804627E60CA8FEF7C3FF0DF22460FEF713
:1087B000BFFF06A8FEF7BCFFB9F1000F07D0D9F83C
:1087C000083023B140460DF2446DBDE8F08F0DF541
:1087D000C660FEF7ADFFF5E76FF00308F2E76FF054
:1087E0000308EFE76FF00308ECE7002070477047DD
:1087F0007047F8B5044615461E460F4621B10830AD
:10880000FEF7D1FF014648BB35B1294604F12C00E3
:10881000FEF7C9FF014608BB36B1314604F1380006
:10882000FEF7C1FF0146C8B9069B33B1194604F1F2
:108830002000FEF7B8FF014680B9079B33B1194607
:1088400004F11400FEF7AFFF014638B94FB104F14F
:108850000800FFF720F86060002001E0A1F58140EA
:10886000F8BD0020FCE7C0F8A410C0F8A8207047AD
:1088700070B504460D461646AC220021FEF733F9CA
:10888000324629462046FFF7EEFF70BDA8B310B56B
:1088900004468C30FEF74CFF04F19800FEF748FFC9
:1088A00004F16800FEF744FF04F12000FEF740FFEA
:1088B00004F13800FEF73CFF04F12C00FEF738FF0E
:1088C00004F11400FEF734FF04F10800FEF730FF56
:1088D00004F18000FEF72CFF04F17400FEF728FF7E
:1088E00004F15C00FEF724FF04F15000FEF720FFC6
:1088F00004F14400FEF71CFF10BD704708B56C2260
:108900000021FEF7F0F808BD2DE9F843DAB306467A
:108910000D461446036803F03F07C7F140081344AF
:108920000360934202D24368013343600FB1444570
:108930000AD23F2C1BD929463046FBF727FD0346B8
:1089400010BB4035403CF4E706F128094246294671
:1089500009EB0700FEF7A3F849463046FBF716FD82
:10896000034688B94544403F3C440027E1E70CB941
:10897000002309E006F12800224629463844FEF784
:108980008EF8002300E000231846BDE8F88370B598
:1089900004460D46036803F03F03581C234480221D
:1089A00083F8282038287CD804F12803C0F1380245
:1089B00000211844FEF797F822686368DB0043EA59
:1089C0005270D1001E0E84F86060C3F3074684F82D
:1089D0006160C3F3072384F8623084F86300C2F354
:1089E000475384F86430C2F3473384F86530C2F3E8
:1089F000471284F8662084F8671004F128012046A5
:108A0000FBF7C4FC0346002859D1E27A2A70A27A07
:108A10006A70627AAA70227AEA70E27B2A71A27B7B
:108A20006A71627BAA71227BEA71E27C2A72A27C63
:108A30006A72627CAA72227CEA72E27D2A73A27D4B
:108A40006A73627DAA73227DEA73E27E2A74A27E33
:108A50006A74627EAA74227EEA74E27F2A75A27F1B
:108A60006A75627FAA75227FEA7594F823202A76B8
:108A700094F822206A7694F82120AA7694F820208F
:108A8000EA76A26EDAB994F827302B7794F826307C
:108A90006B7794F82530AB7794F82430EB77134656
:108AA0000DE004F12806C0F1400200213044FEF739
:108AB0001AF831462046FBF769FC034608B1184610
:108AC00070BD382200213046FEF70DF874E770477C
:108AD00070474FF02002EFF3118382F31188BFF348
:108AE0006F8FFEE710B50446F8F79AFF2046FFF7B0
:108AF000F0FFF8B505460E464FF02003EFF311875F
:108B000083F31188BFF36F8FFCF750FA04463146A8
:108B10002846FFF7E7FF87F31188BFF36F8F2046E2
:108B2000F9F708FFF8BDC26803691A4312F003029F
:108B30000DD10021416105E0416919604361C168BF
:108B40000B44013281689142F6D8002070476FF0E3
:108B500015007047806870470020704790F90E201C
:108B600091F90E309A4201DB0020704701207047D6
:108B700008B5034628B9EFF3058212B9F9F7EEFC00
:108B800003E083F31188BFF36F8F08BD03460068CD
:108B9000834200D070470020FCE738B5054600232B
:108BA0004FF02002EFF3118482F31188BFF36F8F2F
:108BB00043B92846FCF7E0F884F31188BFF36F8FC0
:108BC0000123F5E738BD70B5064600234FF02002BB
:108BD000EFF3118582F31188BFF36F8F1C464BB9F9
:108BE0003046FFF7D3FF044685F31188BFF36F8F3C
:108BF0000123F4E7DCB100234FF02002EFF31185ED
:108C000082F31188BFF36F8F8BB92046FFF7A2FF65
:108C10002146FCF777F8637B23F00203637300239C
:108C2000A36085F31188BFF36F8F0123ECE71CB1BC
:108C300004F1180000F031F8204670BDEFF3058014
:108C4000003818BF0120704708B5F9F783FF08BD49
:108C500038B50446FCF7DCF948B10246206965697D
:108C6000136951691B1845EB010113615161626879
:108C70002368136062685A6000232360636038BD14
:108C800010B5FCF7BBF90446FCF7CEF914B1236923
:108C9000181A10BD6FF00040FBE770B504460023C2
:108CA0004FF02002EFF3118682F31188BFF36F8F2C
:108CB0006FF0150008E02046FFF7CAFF284686F34C
:108CC0001188BFF36F8F01231D461BB92368002B4A
:108CD000F1D1F4E770BD10B500F10C04C46004617B
:088CE000FDF701FB10BD704718
:088CE8004874FF7F0100000049
:108CF000252B0000000000006B6900000000000050
:108D0000AD4C000000000000FD500000000000001D
:108D1000D52A000000000000852100005C00002032
:108D2000113600006C0000208D3900007C0000200E
:108D3000B51F000000000000112300008C0000207F
:108D400013640000000000009171000000000000AA
:108D5000B12F0000AC000020B12F00009C000020CB
:088D600051310000BC000020AD
:108D680000000000012100000000000075690000FB
:108D78006C0000209D3600000000000075690000AE
:108D8800000000007569000000000000756900001F
:108D980000000000E92F00000000000075690000D5
:108DA80000000000756900000000000075690000FF
:108DB80000000000756900000000000075690000EF
:108DC80000000000756900000000000075690000DF
:108DD80000000000756900000000000075690000CF
:108DE800000000007569000000000000A9220000D2
:108DF80000000000756900000000000075690000AF
:108E0800000000007569000000000000756900009E
:108E1800000000007569000000000000756900008E
:108E2800000000007569000000000000756900007E
:108E3800000000007569000000000000756900006E
:108E4800000000007569000000000000756900005E
:108E5800000000007569000000000000756900004E
:108E6800000000007569000000000000756900003E
:108E7800000000007569000000000000756900002E
:108E8800000000007569000000000000756900001E
:108E9800000000007569000000000000756900000E
:108EA8007C000020EF6D00000000000075690000E4
:108EB80000000000756900000000000075690000EE
:108EC80000000000756900000000000075690000DE
:108ED80000000000756900000000000075690000CE
:108EE800FC95000003000000209000000300000033
:108EF8006896000003000000749900000300000059
:108F0800E896000003000000AC9700000100000094
:108F180030950000042700201C9500000100000087
:108F280068950000182700205895000001000000EF
:088F3800FFFFFFFFFFFFFFFF39
:108F40002200000021000000FFFFFFFFFFFFFFFFE6
:108F50000338FDD8704700005374617274696E67FE
:108F600020626F6F746C6F61646572004E52465F71
:108F7000464C4153485F4452565F4E414D450000B8
:108F8000466C61736820646576696365202573208B
:108F90006E6F7420666F756E64000000556E6162BE
:108FA0006C6520746F2066696E6420626F6F7461F7
:108FB000626C6520696D616765000000426F6F74C7
:108FC0006C6F6164657220636861696E6C6F616467
:108FD0002061646472657373206F66667365743AAA
:108FE00020307825780000004A756D70696E672022
:108FF000746F2074686520666972737420696D618E
:10900000676520736C6F74004E65766572207368B7
:109010006F756C6420676574206865726500000078
:109020006D6375626F6F7400696E76616C69642040
:10903000666C6173682049442025643B2065787024
:109040006563746564202564000000000100000071
:109050004093000050940000000000000000000059
:1090600074657374000000007065726D000000008C
:109070004255473B2063616E2774206861707065BC
:109080006E0000007265766572740000537761703F
:1090900020747970653A2025730000005377617061
:1090A00020747970653A206E6F6E650077C295F313
:1090B00060D2EF7F3552500F2CB679800401040343
:1090C0000402040104010403010303040104000079
:1090D0007365636F6E646172790000007072696D10
:1090E00061727900496D61676520696E20746865F9
:1090F00020257320736C6F74206973206E6F742049
:1091000076616C6964210000256420737461747554
:1091100073207772697465206661696C732070656D
:1091200072666F726D696E6720746865207377610F
:109130007000000070616E69632100004661696C17
:1091400065642072656164696E6720736563746F1E
:1091500072733B20424F4F545F4D41585F494D471A
:109160005F534543544F52533D2564202D20746F67
:109170006F20736D616C6C3F000000004661696C8C
:1091800065642072656164696E6720696D616765F9
:1091900020686561646572733B20496D6167653D58
:1091A000257500004661696C6564207265616469BB
:1091B0006E6720626F6F74207374617475733B20E7
:1091C000496D6167653D2575000000004465746563
:1091D0006374656420696E636F6E73697374656E22
:1091E00074207374617475732100000043616E6EA6
:1091F0006F7420757067726164653A206E6F7420B9
:109200006120636F6D70617469626C6520616D6F60
:10921000756E74206F6620736563746F72730000DF
:1092200043616E6E6F7420757067726164653A2079
:109230006D6F726520736563746F727320746861FB
:109240006E20616C6C6F77656400000043616E6E28
:109250006F7420757067726164653A206E6F742058
:1092600073616D6520736563746F72206C61796FD3
:109270007574000062616400676F6F640000000035
:10928000756E7365740000005072696D61727920AB
:10929000696D61676500000025733A206D6167693B
:1092A000633D25732C20737761705F747970653D21
:1092B000307825782C20636F70795F646F6E653D20
:1092C000307825782C20696D6167655F6F6B3D3064
:1092D00078257800426F6F7420736F757263653AFA
:1092E000207072696D61727920736C6F7400000078
:1092F000426F6F7420736F757263653A206E6F6E84
:10930000650000005365636F6E6461727920696D5A
:10931000616765004E6F7420656E6F7567682066C3
:1093200072656520737061636520746F2072756E5D
:10933000207377617020757067726164650000004A
:109340003082010A0282010100D106081A18442C59
:1093500018E8FBFDF70DA34F1FBBEE5EF9AAD24B39
:1093600018D35AE96D188019F9F09C341BCBF3BC63
:1093700074DB42E78C7F10537E435E0D572C44D143
:1093800067080F0DBB5CEEECB399DFE04D840BAAD0
:10939000774160ED152849A701B43C10E6698C2F90
:1093A0005FAC414D9E5C14DFF2F8CF3D1E6FE75B72
:1093B000BAB4A9C8887E473C94C37767544BAA8D3A
:1093C0003835CA62617EB7E115DB7773D4BE7B7234
:1093D00021896924FBF8656E643EC80ED785D55C8B
:1093E0004AE4530D2FFFB7FDF31339833FA3AED2E9
:1093F0000FA76A9DF9FEB8CEFA2ABEAFB8E0FA828E
:109400003754F43EE12BD0D3085818F65E4CC88888
:109410008131AD5FB08217F28A692723F3AB873EB3
:10942000931A1DFEE8F81A246659F81CABDCCE68C6
:109430001B666435ECFA0D119DAF5C3AA7D167C687
:1094400047EFB14B2C62E1D1C902030100010000DA
:109450000E0100003031323334353637383961622D
:1094600063646566000000005B2530386C755D2024
:10947000000000005B253032643A253032643A2522
:109480003032642E253033642C253033645D200067
:109490001B5B306D00000000257300000D0A00000A
:1094A0002530327820000000202020007C000000C1
:1094B0002563000025733A200000000025732E006C
:1094C0003C25733E200000000D0000001B5B313B7B
:1094D00033316D001B5B313B33336D0065727200BD
:1094E00077726E00696E66006462670000000000BB
:1094F000CC940000D49400000000000000000000A4
:1095000000000000DC940000E0940000E4940000FF
:10951000E8940000554152545F3000006C6F675F63
:109520006261636B656E645F756172740000000058
:1095300000000000E51D0000C51D00000000000047
:10954000B51D00009D1D0000FF6400000C270020D9
:109550000A2D0020010000006C6F675F6261636B81
:10956000656E645F7274740000000000E51E000008
:10957000C51E000000000000AD1E0000011E00001E
:10958000611E000024270020202700200100000089
:10959000000000000000000000C000006C8F000010
:1095A0000100000000C00000007006006C8F000089
:1095B0000200000000300700007006006C8F000001
:1095C0000300000000A00D0000E001006C8F00000F
:1095D0000400000000800F00008000006C8F00007D
:1095E000050000006866636C6B0000006C66636CCD
:1095F0006B000000434C4F434B000000636C6F63F3
:109600006B5F636F6E74726F6C000000A96800007E
:10961000596800009F6800000000000059670000C2
:109620002920000055210000E4950000D11F000012
:10963000DD1F0000EC950000C9200000A9200000FB
:10964000000000007379735F636C6F636B00000050
:109650005465726D696E616C0000000052545400D4
:1096600053454747455200006D7075004661696C6F
:10967000656420746F20616C6C6F63617465206E2B
:109680006577204D505520726567696F6E2025758E
:109690000A000000506172746974696F6E2025754C
:1096A0003A2073616E69747920636865636B206624
:1096B00061696C65642E0000464C4153485F300080
:1096C0005352414D5F30000002000000D096000070
:1096D00000000000B89600002600020200000020F2
:1096E000C096000022000B11736F63004750494F72
:1096F0005F3100004750494F5F3000006D2B000084
:109700002F6B00003D6B0000536B00005F6B00008F
:109710006B6B0000FD2E00007D6B00000000000060
:10972000FFFFFFFF0000005000000000FFFF0000EF
:1097300000030050010000003D6D0000DD6C0000E2
:10974000356C0000E16B0000493100003931000048
:1097500004000000FF000000053300009135000008
:109760003533000045330000DB6D0000ED330000B1
:109770001D3400003D3500005934000085340000E0
:10978000653400007534000085340000B9340000F1
:10979000C9340000D9340000E9340000EB6D00004A
:1097A00029350000554152545F31000075617274D3
:1097B0005F6E7266785F7561727465000B6F000092
:1097C00095700000FD6E00003D6E0000ED6E000023
:1097D0003D6F00008F6F0000BB6F0000D16F000075
:1097E000DB6F00001770000023700000DB6F0000CB
:1097F000077000002F7000003D7000004B700000EB
:1098000085700000897000000080024000000000A8
:10981000982F8A4291443771CFFBC0B5A5DBB5E9DB
:109820005BC25639F111F159A4823F92D55E1CAB4F
:1098300098AA07D8015B8312BE853124C37D0C55DD
:10984000745DBE72FEB1DE80A706DC9B74F19BC125
:10985000C1699BE48647BEEFC69DC10FCCA10C2415
:109860006F2CE92DAA84744ADCA9B05CDA88F976F9
:1098700052513E986DC631A8C82703B0C77F59BF63
:10988000F30BE0C64791A7D55163CA06672929148F
:10989000850AB72738211B2EFC6D2C4D130D38532C
:1098A00054730A65BB0A6A762EC9C281852C7292EE
:1098B000A1E8BFA24B661AA8708B4BC2A3516CC71C
:1098C00019E892D1240699D685350EF470A06A1055
:1098D00016C1A419086C371E4C774827B5BCB034A4
:1098E000B30C1C394AAAD84E4FCA9C5BF36F2E6842
:1098F000EE828F746F63A5781478C8840802C78CD1
:10990000FAFFBE90EB6C50A4F7A3F9BEF27871C6D3
:10991000F08C0000388D0000408D0000688D000044
:10992000688D0000F5FFFFFF7A65706879722D760B
:10993000322E332E302D313937312D673265643276
:109940006433626661396263000000002A2A2A20BB
:10995000426F6F74696E67205A6570687972204F24
:1099600053206275696C64202573202573202A2A90
:089970002A0A00006F730000D9
:10997800FFFFFFFFDD5B0000E9630000909500003A
:10998800216B000000C2010000010300000000007C
:1099980000000000A82C00202000000000C20100E8
:1099A800000103001C00002000000000000000006F
:1099B8000090D003EB870000F1870000EF870000DC
:0C99C800E76A000054000020540000205A
:1099D400F4950000209600000C9600004427002017
:1099E40014950000000000005897000014000020A7
:1099F400A497000008980000BC9700002C000020E9
:109A04004496000000000000000000000000000078
:109A1400F496000020970000FC960000582C0020CB
:109A2400EC9600002C970000FC960000742C00209B
:109A34006C8F000000000000389700000000000058
:109A4400CC000020CC00002000000000000000003A
:109A5400FFFFFFFFE0000020E00000200000000006
:089A640000000000FFFFFFFFFE
:109A6C00F4000020F40000200000000001000000C1
:04000003000026F1E2
:00000001FF
